:020000041000EA
:1004000000C00E08EB0400100D0000004D050010A8
:1004100000000000000000000000000000000000DC
:10042000000000000000000000000000490500106E
:100430000000000000000000490500104905001000
:100440004905001049050010490500104905001034
:100450004905001049050010490500104905001024
:100460004905001049050010490500104905001014
:100470004905001049050010490500104905001004
:1004800010B5064C2378002B07D1054B002B02D06A
:10049000044800E000BF0123237010BDF0050E08E2
:1004A0000000000064720010044B10B5002B03D054
:1004B0000349044800E000BF10BDC0460000000032
:1004C000F4050E08647200100230800803D0013079
:1004D0000238FCD1C046C0467047EFF3108072B6B8
:1004E000704780F3108870477047FFF7FDFF72B6C2
:1004F0000F4C104DAC4209DA21686268A368043BD6
:1005000002DBC858D050FAE70C34F3E70A490B4A2B
:100510000020521A02DD043A8850FCDC08480949E0
:100520000860BFF34F8F05F0A3FF05F02DFFFEE736
:100530007072001088720010F0050E08B00B0E08E3
:1005400000000E0808ED00E0FEE7FEE700B504201D
:100550007146084202D0EFF3098001E0EFF3088012
:10056000043005F06BF9FEE70300093B0122042B80
:1005700002D920384242424110007047F0B50025B0
:10058000170006002C0089B003930E9B02901B0CF1
:10059000DBB204930E9B00911B0ADBB205930E9B0A
:1005A000DBB20793731C069333780193002B08D0BA
:1005B000009B002B22DB029A731C9B1A009A9A4222
:1005C0001CDA0E9BDBB2002B00D1B4E0019A9A42F8
:1005D00000D0AEE0009B002B06DB029A731C9B1A36
:1005E000009A934200DDA4E0B31C7678032D00D975
:1005F000A1E0280005F0DCFF8989637B0198FFF703
:10060000B3FF002839D1079B019A9342D9D04F4EAE
:100610001100300006F098FA031E08D1049B019ADD
:1006200093420BD0059B93426FD133003F33032D90
:1006300023D8280005F0BCFF0510233533003E33D6
:10064000F5E7002F06D0039A94425ED23F4A9B1AE8
:100650009B003B55012510E0621C002F0BD0039935
:100660008A4252D239493C195B1A21781811014348
:100670001B012170BB5414000225069E92E7621CE8
:10068000002F0BD003998A423FD230493C195B1AA4
:100690002178981001439B012170BB54140003255D
:1006A000EBE7002F08D0039A94422ED227493A193B
:1006B0005B1A11780B43137001340025DDE71D0030
:1006C000002E22D0009B002B22DB029B009AEB1A0B
:1006D0009A421DDA019BB34217D1009B002B04DD27
:1006E000029B009AEB1A93420FDC2E786B1C029A45
:1006F0009D1A002E04D0009B002B11DBAB420FDAB9
:10070000002F18D03B5D002B15D00124644219E066
:100710003000FFF729FF0028DCD02E780135CFE725
:100720003000FFF721FF0028EFD0029B5E5D01350E
:10073000DFE7002DE9D1039B9C42E6D2002F01D0D8
:1007400000233B55200009B0F0BDC046A06D00104D
:10075000002210B504001000A15C0B00303B092BF7
:1007600009D830380818531C032A03D000011A0096
:10077000042BF1D110BD0B00413B052B01D83738BC
:10078000F0E70B00613B052B01D85738EAE7002062
:10079000F0E70000F0B50B7885B0039017004D1C12
:1007A000222B17D0116000202AE05C2A07D1019A81
:1007B0005278002AF7D0019A013301320192019A4E
:1007C00001320192019A1278222A00D1A7E0002A70
:1007D000EBD1E8E701950023F4E72B785C2B11D0EF
:1007E000237001350134019B9D42F6D30023039A07
:1007F00023700833D36013000198029A01301A6104
:1008000005B0F0BD6B78662B63D014D82F2B61D068
:1008100007D8222B5ED0484B3D601B680298984752
:10082000C1E75C2B56D0622BF5D10823237001342D
:10083000063BED18D7E7722B50D006D86E2BEAD1C5
:100840000A2323700134083BF3E7742B48D0752B3F
:10085000E1D1019B5B1B052BDDDDA81CFFF778FFB9
:10086000364B374AC31806009342D4D90028D2D059
:10087000344B334AC318934234D8019AAB1DD31A70
:10088000052BC8DDAB795C2BC5D1EB79752BC2D1BB
:1008900028000830FFF75CFF284B294AC318934211
:1008A000B9D8294BB6021E4080238005800D5B021B
:1008B0000643F6180C23254A96421FD9244A96422D
:1008C000A9D83F203040802676420643E6700422B5
:1008D00012E00C23237001340223AAE70D23F9E769
:1008E0000923F7E77F2804D91A4B98420ED906232B
:1008F000E1E7062301222070A4189AE73F20304048
:10090000802676420643A6700322F5E73F20802327
:1009100006405B421E43667086330222ECE7019A72
:10092000501AC01A0C4B04301B6898470290041EE2
:1009300000D058E737E7C04680000E080024FFFFCC
:10094000FF0300000028FFFF00FC0F00FFFF000076
:10095000FFFF1000FF07000084000E08002803D0EE
:100960000378013B1F2B00D970470130F6E70000E8
:10097000064B10B51B6828209847041E03D0282278
:10098000002106F01EF8200010BDC04684000E08AD
:100990000849094A002803D1084B0B60084B07E0BF
:1009A0000368002B00D1054B0B604368002BF5D08A
:1009B0001360704784000E0880000E0865690010FF
:1009C00079690010F8B5802604007600002C00D16B
:1009D000F8BDE3682768334204D1A068002801D03D
:1009E000FFF7F0FFE3680B4D334204D12069002884
:1009F00001D02B6898478022E3689200134204D10B
:100A0000206A002801D02B68984720002B6898475F
:100A10003C00DBE780000E08F0B5040085B00F0055
:100A20001600002901D1002013E004226F4938008C
:100A300006F0AAF8002803D10223E360381D08E07D
:100A400005226B49380006F09FF8002803D1E060CA
:100A5000781D05B0F0BD04226649380006F094F810
:100A6000002806D101230122E3600023A261E36193
:100A7000E4E73B78222B05D1320039002000FFF754
:100A800089FEE6E72D2B03D01A00303A092A24D834
:100A900000250A2203A93800039506F033F9030064
:100AA00003988742BFD05A1C0AD1534A914211D1B0
:100AB0000122514B5242A261E3610423E360C8E783
:100AC000002B07D180221206914203D180230022FD
:100AD0001B06F0E7A361E161EFE75B2B35D1781CE2
:100AE000FFF73CFF037805005D2B26D00023013D76
:100AF00001930093FFF73CFF009B071E6FD0002B74
:100B000019D0019B18604360681CFFF727FF320073
:100B100001003800FFF780FFFFF720FF051E06D019
:100B2000037801972C2BE5D05D2B08D0306000981E
:100B3000FFF748FF77E70090E6E7002300931023D4
:100B4000E360009B681CA36083E77B2B4BD1781C80
:100B5000FFF704FF037807007D2B38D00023013F07
:100B600001930093FFF704FF009B051E37D0002B75
:100B700017D0019B18604360781CFFF7EFFE32002E
:100B800001002800FFF706FEFFF7E8FE0028CED0A0
:100B90002B692B6200232B6103783A2B03D0306042
:100BA000C5E70090E8E70130FFF7D8FE320001000A
:100BB0002800FFF731FFFFF7D1FE071EB7D00378FB
:100BC00001952C2BCED07D2B03D03060AFE70023D6
:100BD00000932023E360009B781CA36039E7002B7F
:100BE00000D120E7A3E737601DE7C046DF6D0010A6
:100BF000E46D0010EA6D0010FFFFFF7FF7B5050000
:100C00000E0001920F1E00D1144FFFF7B1FE00231A
:100C100004003B6098420DD02800FFF79FFE3A0089
:100C200001002000FFF7F8FE051E05D12000FFF7A8
:100C3000C9FE00242000FEBD019B002B0AD0FFF757
:100C40008DFE03780500002B04D02000FFF7BAFECC
:100C50003D60EEE7002EEDD03560EBE70C060E08A8
:100C6000002210B51100FFF7C9FF10BDF0B58DB01F
:100C70001D0012AB40CB02921B780F0003930023A0
:100C800006AA05A90593069300F021F9041E3FD199
:100C9000224B3A0000930699029B0598FFF76EFCE1
:100CA000002838DD022008AA07A9FF30079408941D
:100CB00000F0CAFE002802D06524644228E0290022
:100CC000079800F0E7FC0028F6D1033008AA07A92E
:100CD000FF3000F0B9FE0028EED13100079800F097
:100CE00077FC041E14D109A9380000F008F9041E8D
:100CF0000ED131000A9800F0C7FB041E08D1039AF8
:100D000029000B9800F01AF904000998FFF75AFE21
:100D100020000DB0F0BD1424CFE7C046005F2D00C9
:100D2000F0B51F00002387B00291039204A905AA21
:100D300006000493059300F0CAF8041E1ED105981E
:100D400000F068F8040005F00DFE051E1CD0104BE5
:100D500002000093059923000498FFF70FFC002878
:100D60000FDD039B220000930197029B29003000B6
:100D7000FFF77CFF0400280005F0FEFD200007B00F
:100D8000F0BD14246442F6E764246442F6E7C046EA
:100D9000005F2D0010B5010004000B4805F0E2FED5
:100DA000002398420DD02100084805F0DBFE012306
:100DB000002806D02100064805F0D4FE43424341F6
:100DC0005B00180010BDC046DE6E0010E76E00101C
:100DD000EF6E001010B5010004000B4805F0C2FED4
:100DE000002398420DD02100084805F0BBFE0123E6
:100DF000002806D02100064805F0B4FE43424341D6
:100E00005B00180010BDC046C46E0010CD6E00100F
:100E1000D96E00100323584380089843043070476C
:100E2000F8B5C3680D000860202B19D184680E4FF7
:100E3000002C01D12000F8BD266A002E06D031001A
:100E40000A4805F08FFE002802D16C602468EFE7A5
:100E50003100380005F086FE0028F7D1AC60F5E7D8
:100E600002204042E7E7C046FD6E0010F76E00101A
:100E7000F0B507000D00002491B001AE002D02D1A5
:100E8000280011B0F0BD296A002904D0380005F00F
:100E900069FE0028F4D0AB68002B06D00E2C12D8C7
:100EA000A200955101341D00E8E72B68002BFAD110
:100EB000002C0AD0013CA3009B591B68002BF2D1E7
:100EC000002CF7D1EFE70025DAE72500D8E7F8B5E1
:100ED0000E002E21170005F037FE041E0CD0451C15
:100EE0002E21280005F030FE002805D0001B013817
:100EF000386000203560F8BD16204042FBE770B531
:100F0000050000200C00FFF743FD2800FFF7A8FEB6
:100F1000002803D02100FFF783FF70BD0520404269
:100F2000FBE7002304220133002901D1904203D9B9
:100F300052001D2BF7D1023318007047F0B589B06D
:100F400005900C000100C6480792FFF791FF0028AA
:100F500000D11FE283680193029300231F000693D0
:100F60000493029B002B42D1019BDB680293202B50
:100F700000D010E2019D2900BA48FFF779FF061E54
:100F800000D198E0037E079A9A4200D093E00100D6
:100F9000B548FFF76DFF002800D189E08369237011
:100FA0003100B248FFF764FF1423002800D08369A2
:100FB0006360002F00D0EEE1019E3100A948FFF7E9
:100FC00057FF00287CD02278037E9A4278D13100E6
:100FD000A748FFF74DFF002800D1FCE028238269D5
:100FE000551E6B43E3181A74022302936FE00299B3
:100FF000A048FFF73DFF002802D08668002E03D1ED
:10100000029B1B680293ACE731009B48FFF730FF5F
:1010100000284BD0036999491800039305F0A2FDFD
:10102000002843D09649039805F09CFD00283DD048
:101030000025944AAB009958039805F093FD071ECC
:1010400005D00135172DF4D10527183D7F42310019
:101050008D48FFF70DFF002801D08369069331000A
:101060008A48FFF705FF002804D0C1698069FFF7AF
:1010700058FF04906B1C19D0049B002B16DDAD2388
:101080006A00A2185B00D35C012B05D12B000F3343
:10109000DB000699E31859605C23FF33D35C012B16
:1010A00004D10F35ED00049B6519AB603668A5E7E8
:1010B00001277F4274E72D68002D00D05BE778E7B9
:1010C0003668002E00D078E7012335000293002E09
:1010D00000D084E031006E48FFF7CAFE002800D03F
:1010E0000FE131006B48FFF7C3FE00280ED00D233F
:1010F0006B43E3183633FF331B78012B06D1C268EC
:101100002733511E8A416B43E3185A7031006248FD
:10111000FFF7AEFE00280ED00D236B43E3183833E3
:10112000FF331B78012B06D1C2682733511E8A4139
:101130006B43E3181A7231005848FFF799FE0028F4
:101140000CD00D236B43E3183833FF331B78012B8E
:1011500004D127336B438269E3185A723100504837
:10116000FFF786FE00280FD00D236B43E3184133B1
:10117000FF331B78012B07D1C2682733511E8A41E8
:101180006B43E3180833DA7731004648FFF770FE07
:10119000002800D1C5E0C368102B00D0C1E08268F0
:1011A0000D211B2000236943684361180390002A26
:1011B00000D1B6E01F003E37FF37CF5D012F04D1CD
:1011C00003981F1890692437C8550133032B00D1A9
:1011D000A7E01268EBE701230500029377E73100EF
:1011E0002448FFF745FE002800D173E78768002FE9
:1011F00000D16FE739002048FFF73AFE00282DD0D4
:1012000003691E491800039305F0ACFC00284BD17C
:1012100039001D48FFF72CFE00280CD00D236B432E
:10122000E3183A33FF331B78012B04D127336B4388
:101230008269E3185A6139001448FFF719FE002843
:101240000CD00D236B43E3183B33FF331B78012B8A
:1012500004D127336B438269E3189A613F68C6E77C
:10126000C46E0010656E0010136E00101A6E001030
:10127000226E0010EF6D00100A6F0010F96D001063
:10128000FE6D001088000E08066E00100E6E001035
:101290002E6E0010026F0010386E0010406E0010AD
:1012A0004F6E0010566E00106B49039805F05AFC03
:1012B0000028D3D139006948FFF7DAFD00280CD0A7
:1012C0000D236B43E3183C33FF331B78012B04D110
:1012D00027336B438269E318DA6139006048FFF70E
:1012E000C7FD0028BAD00D236B43E3183C33FF330E
:1012F0001B78012BB2D127336B438269E3181A6242
:10130000ACE70D236B43E3183933FF331B78012B14
:1013100000D0E6E627336B438269E318D2B2DA6085
:10132000DFE631004F48FFF7A3FD28236B43E318A6
:10133000002829D082699A70002D08D131004A48CE
:10134000FFF796FD1423002800D08369E362029B17
:10135000022B1FD1019E31004448FFF789FD002870
:1013600014D08269D3B2022B10D12827551E6F43A7
:10137000E219137431003E48FFF77AFD002801D0CE
:1013800083693B55012330E69870D5E73668002E17
:10139000E1D1F7E7002705993648FFF769FD0028F6
:1013A0002ED0002F2CD13D008668002E28D0310091
:1013B0002B48FFF75DFD00280BD063191A0050324F
:1013C000FF321278012A04D102326A439B188269E3
:1013D0005A6531002848FFF74BFD00280BD06319F0
:1013E0001A004F32FF321278012A04D102326A43C6
:1013F0009B1882691A6502350A2D01D03668D4E738
:1014000005991E48FFF734FD051E22D0002F20D17C
:1014100001001B48FFF72CFD00280AD05A23FF3398
:10142000E35C012B05D1C3685A1E93412200793237
:10143000137029001348FFF71BFD002809D0AC23C7
:101440005B00E35C012B04D1C36878345A1E9341DE
:101450002370380009B0F0BDFE6D0010066E00105C
:101460000E6E0010606E00101A6E0010226E0010DA
:10147000656E0010686E0010726E0010786E0010BD
:10148000846E0010906E001070B50C0001001648BC
:10149000FFF7EEFC051E24D001001448FFF7E8FC1E
:1014A000002806D0E378012B03D10069FFF772FC16
:1014B000207029000E48FFF7DBFC002806D02379B6
:1014C000012B03D10069FFF785FC607029000948F2
:1014D000FFF7CEFC002804D06379012B01D183698A
:1014E000A370002070BDC046A26E0010A56E001053
:1014F000B06E0010B86E001070B504000D0086B01C
:101500000021142201A805F05CFA29002000FFF751
:10151000AFFC0400002C18D021001C48FFF7A8FCE9
:101520000028F7D00569002D0AD0194E2900300097
:1015300005F018FB00280BD1310001A805F01CFBB9
:10154000210001A8FFF794FC0400200006B070BD44
:10155000104E2900300005F005FB0028ECD02900D2
:101560000D4805F0FFFA0028E6D00C4E29003000A7
:1015700005F0F8FA0028DFD02900094805F0F2FA52
:101580000028DDD121000748C1E7C0460A6F0010DE
:10159000326F00101B6F0010226F00102A6F0010B6
:1015A0000F6F0010156F001010B5FFF761FC0124DC
:1015B000002809D08168002906D00448FFF758FCAC
:1015C000002801D0C468E4B2200010BDBC6E001039
:1015D000F7B5040000200D00FFF7DAF92000FFF74F
:1015E0003FFB071E4AD001002648FFF741FC041EBE
:1015F00006D1012676423800FFF7E4F93000FEBD3F
:1016000001002148FFF778FF210006001E48FFF780
:10161000CBFF0090002E2BD03069FFF7BBFB6B4651
:1016200000261B782870EB7021001848FFF764FF34
:10163000210000901548FFF7B7FF009B0190002B99
:1016400019D01869FFF7C6FB6B461B7968702B71C0
:1016500021000F48FFF750FF210000900C48FFF7D2
:10166000A3FF009B002BC4D09B696871AB70C2E7DD
:1016700001267642D8E701267642E9E7052676423A
:10168000BCE7C046A26E0010A56E0010B06E001040
:10169000B86E0010F0B5050085B000200C00FFF713
:1016A00077F92800FFF7DCFA0190002800D1A8E1C3
:1016B0000100D648FFF7DCFB051E00D161E1D44FE5
:1016C00001003800FFF718FF290006003800FFF777
:1016D0006BFF002E00D134E19A22B3695200DBB2D5
:1016E0002370A0542200283213704223FF33E054A9
:1016F0000023C84F290038000093FFF7FDFE2900A2
:1017000006003800FFF750FF002E00D11CE1F368FF
:101710005A1E93413622DBB2FF326370A05422007E
:1017200029321370A1235B00E054BB4F290038001D
:10173000FFF7E2FE290006003800FFF735FF002E14
:1017400000D105E1F3685A1E93413822DBB2FF3223
:101750002372A054220030321370A2235B00E054A5
:10176000AE4F29003800FFF7C7FE290006003800F9
:10177000FFF71AFF002E00D1EEE09C22B369520061
:10178000DBB2E360A05463634623FF33E054A44F0D
:1017900029003800FFF7B0FE290006003800FFF7E7
:1017A00003FF002E00D1DBE0B369621DDBB2D3770B
:1017B0003E22FF32A05422004C321370A522520068
:1017C000A054A21DD3779F225200A05422004D3274
:1017D00013704C22FF32A054E21DD3774022FF3217
:1017E000A05422004E321370A6235B00E0548D4EAD
:1017F00029003000FFF780FE290007003000FFF7C6
:10180000D3FE002F00D1AFE0FB685A1E93412200A7
:10181000DBB20832D377A0225200A05422004F320C
:1018200013704E23FF33E05401997F48FFF720FBEC
:101830000600002F00D1A4E03A220123FF32A35476
:10184000D218A3543C22FF32A354D218A35402232B
:10185000764FFF330A32A35202320100A3523800FE
:10186000FFF74AFE310005003800FFF79DFE0390A8
:10187000002D00D17CE0AB6902936D4F3100380040
:10188000FFF73AFE310005003800FFF78DFE002D0E
:1018900000D172E0AD692200210023005B323531B6
:1018A0007C33FF32FF31029E5D601E606E46367BE8
:1018B00008331670507002328B42F4D101995D48A2
:1018C000FFF7D6FA061E69D05B4F01003800FFF71C
:1018D00013FE310005003800FFF766FE0390002D6F
:1018E00053D0AB690293524F31003800FFF704FE2A
:1018F000310005003800FFF757FE002D4AD0AD69D2
:101900002200230021004F325033FF327831029EF3
:101910005D601E606E46367B083350701670023272
:101920009942F4D101994548FFF7A2FA051E39D131
:1019300001235B4200930198FFF744F8009805B03B
:10194000F0BD01235B42D4E601235B420093ECE649
:1019500001235B42009303E701235B42009316E7F8
:1019600001235B42009342E701235B4200935BE764
:1019700001235B42029500937FE701235B420093C2
:1019800089E701235B42009398E701235B420295BC
:101990000093A8E701235B420093B1E701235B4278
:1019A0000093BFE7264F01003800FFF7A5FD29008F
:1019B00006003800FFF7F8FD002E1ED0F3685A1E0F
:1019C0009341220078321370AC235B00E0541D4F2A
:1019D00029003800FFF790FD290006003800FFF7C6
:1019E000E3FD002EA4D0F3685A1E93412200793201
:1019F00013705A23FF33E0549DE701235B420093A9
:101A0000E5E705235B42009398E7C046C46E0010EB
:101A1000656E0010026F0010386E00102E6E001000
:101A2000566E00104F6E0010EF6D0010066E001025
:101A30000E6E0010686E0010726E0010786E00104E
:101A4000906E0010846E0010DC23F0B59B0585B00D
:101A50000093002302AD019502901848184C0668C7
:101A60006B60306A0768002F07DBA34203D10120B7
:101A7000404205B0F0BD0133F4E7A342F7D06B4616
:101A8000C3600123B03683603368C0180023066842
:101A9000002E03DAA342EAD00133F8E7A342E6D0EE
:101AA000A02300981B06984201D00098E1E7029B12
:101AB000002013606B680B60DBE7C04618090E0856
:101AC000983A00000122F0B50024184B0668196806
:101AD00032400B6AB0310D6815495D191F68002F3F
:101AE00006DB8C4202D101204042F0BD0134F5E713
:101AF0008C42F8D0002A00D106000120DE609860F8
:101B000000202C68002C03DA8842ECD00130F8E782
:101B10008842E8D0DB68002A00D11B68A0220020A0
:101B200012069342E1D01800DFE7C04618090E08FC
:101B3000983A00000A4B37B51B780500013B00249A
:101B4000012B05D8074B01A80193FFF7BBFF040049
:101B5000002D02D0280003F02BFE20003EBDC04621
:101B6000A40B0E080101013A07B5034B01A801932C
:101B7000FFF7A8FF0EBDC0460101003210B5FFF708
:101B8000F3FF002801D105F0FBF810BD70B504008B
:101B90001000FFF7CFFF174B1B68002B23DA8023C1
:101BA000154A16499B00D1501549164E0968080080
:101BB00090300D680068281805682E40124D354396
:101BC0000560080015008830096800681E00F13BB8
:101BD0000918FF3B0A681A42FCD0012003F0E8FD17
:101BE000AC51FFF7CBFF200004F0BCFC002004F058
:101BF000CDFAFBE70001264000002040004000161F
:101C000018090E08FCFF00000300FA05014B1860DC
:101C10007047C04618090E08044B1B681A00AC3206
:101C200012881B6A5043C0187047C04618090E0836
:101C30001D4B98420FD010D840282FD005D800282F
:101C400030D0102828D019481EE0802828D08023C2
:101C50005B009842F7D1144816E0154B984214D017
:101C600008D8A0231B0698421CD0124B9842EAD1F8
:101C7000A0200BE0104B98420AD0104B984209D09C
:101C80000F4B9842DFD10F487047A420C003FBE7F9
:101C90000D48F9E70D48F7E70D48F5E70D48F3E77C
:101CA0000D48F1E70020EFE706005200FF00520068
:101CB000010000F0090000A0040000F0050000F0A1
:101CC000030000F001005200020052000300520025
:101CD00001005000020050000500520010B5002025
:101CE000FFF79AFF0A4B1C682300B0331B68C0182B
:101CF0000368002B0ADB074B1868FFF799FF0122E6
:101D000063689A609A68002AFCD110BD0248FCE71B
:101D100018090E0810060E08020050000E4B10B5F0
:101D20001B689C695B69001BC0090001C0181F2368
:101D30001A40032907D8C9008B408A4004689C4395
:101D40002243026010BD0439C9008B408A404468B8
:101D50009C4322434260F5E718090E08F7B50126B7
:101D600037008F4033408B4005681400BD430F2778
:101D70002B4303600A4B08AA12781B68019279333F
:101D80001D788E0045192B683C401A003B00B3407B
:101D9000B4409A4314432C60019AFFF7BFFFF7BD8C
:101DA00018090E08064B1B68B0331B68C3181B6864
:101DB000002B03DA89B24160002070470148FCE73C
:101DC00018090E0801008A000368002B04DA89B2A2
:101DD000C2608160002070470048FCE701008A0073
:101DE000064B1B68B0331B68C3181B68002B03DA53
:101DF000C36800200B6070470148FCE718090E0813
:101E000001008A00024B1A68002A00D1186070474E
:101E100024060E08F0B52C246043124C1F002468E1
:101E20001E0A2018FF24274034400F4E1B0C356833
:101E300007602E6A44608360AC352D8880346F4320
:101E400064013419BF191E04334307614461A36060
:101E500000238361059BC2610162002B01D01B88B6
:101E60008381F0BD24060E0818090E08F0B58368BA
:101E700085B002AD2B80154B02681B68066A9B8EED
:101E8000476A9B186B8043680095826AC16A0400A8
:101E900003930369C068FFF7BDFF00213B000A0000
:101EA00000913000FFF7B6FF216B280003F036FCED
:101EB0000022AB5E002B06DB1F2213401E3A9A4025
:101EC0001300034A136005B0F0BDC04618090E08A0
:101ED00000E100E0F7B52C25134C68432668694300
:101EE0003418256901937118002D19D088690028CC
:101EF00018D12E68002E15DA6768012426004B6879
:101F00009E40B44613689EB263461B041E4316608F
:101F1000EA608C61BC40019BA4B24B62AC60FEBD28
:101F20000248FCE70248FAE724060E0804028A0089
:101F300007028A0073B5002642690400D56801963D
:101F40002B0CB34221D01B0413601368194B00699A
:101F50001B68B0331B68C3181B68B34215DA01A9AC
:101F6000FFF73EFFB0420CD10198E26903681E0CF6
:101F7000DBB29A4205D9226A9B009B58002B00D005
:101F8000984731002069FFF70DFFADB2002D09D051
:101F900063691D6000251B68636AAB4205D09847E2
:101FA0006562A56163691B6873BDA36A002BF8D0E5
:101FB0009847F6E718090E082C2310B54343034A47
:101FC0001068C018FFF7B6FF10BDC04624060E0803
:101FD000F8B5194B0F001B681A002E321278824296
:101FE00027D9002925D01F250A68154021D11900BD
:101FF000AC310C88114E60431C6AD20804192900C8
:102000007868346004F0DDFC29002000FFF7CAFE88
:102010003A0029003068FFF7D7FE041E07D10100FF
:102020003068FFF7BFFE03002000002B00D00448FB
:10203000F8BD0448FCE7C04618090E0828060E083B
:1020400001018A0003018A0010B5002A0DD1002980
:1020500014D10B4B1A681300AC331B885843136A16
:10206000C018084B1860080010BD002906D0064BA8
:10207000196019005A60FFF7ABFFF5E70348F3E773
:1020800018090E0828060E080400000803018A003B
:10209000F7B5184F04003B680191DE68336883424E
:1020A00026D90025A94202D1FEF717FA05003868A3
:1020B0000368002B1ADA1F2201232240934064098F
:1020C0007268A4001419226813420DD09A4322604A
:1020D00000240021FFF766FE019B002B02D128009F
:1020E000FEF7FFF92000FEBD034CF2E7034CF3E7D7
:1020F000034CF7E728060E08020188000301880058
:1021000004018A000A4B1B68DB681A6882420DD9F9
:1021100059681F23420918401E3B834092005058C3
:102120001840431E9841034BC01870470248FCE713
:1021300028060E080001880004018A0070B50F4BC4
:102140001B683B331A78431E591E8B419A4213D9A0
:102150000B4B0C4D8000C41863590B4A01201A40E8
:1021600080239B051343635103F03CFB002063591C
:102170005B005B08635170BD0448FCE718090E085A
:1021800000002640FC050000FFFFFFCF01004A00D1
:10219000F7B59621002003F069FB4C4E4C4C336898
:1021A0001A003C321278002A00D188E00027E02192
:1021B00030203D0089006258824362501A001900A5
:1021C000083201C9D26F01918218106841498C46CA
:1021D0000840019910601A68C96F50188021026880
:1021E00049041202120A0A4361460260019A1B68FE
:1021F000D26F9B181A680A401A6004F0F7F8336827
:102200003B331B78002B03D00120FFF797FF07001B
:10221000002F00D0304D33683B331B78012B03D99E
:102220000220FFF78BFF0700002F00D02B4D00216D
:10223000012002F09FFE002800D0294DE0270F2347
:10224000BF00E059184012D102F0BCFE1223FF3348
:1022500098420CD133683C331B78002B32D00F23CB
:10226000E2599A430E3B1343E35104F0BFF8B12106
:10227000C90063581B4A1A4080239B051343B022B0
:1022800063500021D200A35808005B005B08A350F4
:10229000154AA3585B005B08A35002F06BFE0028B0
:1022A00000D0124D33683C331B78002B0CD0E02259
:1022B0000F219200A3588B43A3502800FEBD0C4F62
:1022C0000C4D7BE70B4DD0E70A4DF6E718090E08D9
:1022D00000002640FF00FFFF2F0F1A012E0F1A01EA
:1022E0004E0F1A01FFFFFFCF8C0500004F0F1A01A0
:1022F00001004A000F0F1A01BE4BF0B51B6887B0F2
:102300001A00AC321188186A8A001218D06802903C
:102310000088059002984088009002988768C068FD
:10232000049005980138072809D804F04BF9620099
:1023300026004500D4087E00C60052027100AE4C53
:102340006A46029B928A85211A806A4680201288FA
:102350005C605A80049A9F60DA60A64B49011B6852
:1023600040031A6AAC3350501888515880008018C6
:102370000021FFF717FD07B0F0BD009A9F4BD20078
:1023800099184968049C0C4001D001F0A7F8481C3A
:1023900001D101F0A6F800981F2801D901F0A4F896
:1023A000D258002A01D101F0A2F8136839430B403A
:1023B00004990B431360C3E73C00009A8F4BD20093
:1023C000991849680C4001D001F094F8481C01D1DB
:1023D00001F093F800981F2801D901F091F8D25824
:1023E000002A01D101F08FF813680B403B431360C2
:1023F000A6E7009B1F2B01D901F088F8DA007F4B7C
:10240000D358002B01D101F084F81F68002497E70E
:10241000022F01D001F080F8049C63425C41784BAC
:1024200064421C40774BE4188AE7002F01D101F089
:1024300076F8754CF0223900200004F0B9FA03F068
:10244000EDF9002810D0FFF7A3FE6F4801F002FC61
:102450006E4B04001A78002A00D071E7002800D0E3
:102460006EE701321A706BE7684B1B78002BECD1DA
:10247000E378002BE7D0E379002BE4D055342478BF
:1024800003F0BAF90028DED1614B624A995800295D
:1024900008DAC02149005958C907D4D499584900CD
:1024A0004908995080219858090601430120995004
:1024B000995881430C439C50C5E70098662835D055
:1024C00017D82F2800D174E106D82C285BD02D28EE
:1024D00000D1D4E0484C33E7009B302B00D16DE1B4
:1024E000322BF7D13A893888796802F0D5FF040099
:1024F00026E700986D2800D13BE107D8672833D044
:102500006C28E7D103F0BAFB002419E7009A6E2A81
:1025100000D139E16F2ADDD13878072801D901F0DF
:1025200001F8797803F0C8FB002409E7384B5A68B2
:10253000002F10D1384911401B220A435A605968B4
:10254000364A1143596059681143596059680A4322
:102550005A600024F4E6E821314889010240114321
:1025600059605A680240F3E703234B439B181A68EB
:10257000002AFCDA80220024D96852050A43DA6076
:102580005C605B68DCE60024B126264BF6001C800C
:10259000254B1C80174B1B683B331B789C4201D991
:1025A0000024CDE61A4D002C1ED1B023DB00EB58E1
:1025B000DB0F17D0200002F005FD022855D1002CBA
:1025C00036D18020AB59194A800513401843A851D1
:1025D0000021200002F0CEFC0123A340114A118803
:1025E0000B4313800134D5E723008033FF339B0076
:1025F000DDE7C04618090E08FF0F1A011C090E0876
:1026000007F0E5FEF90F1A0130060E0820070E0844
:10261000000026400C0500000000FC0F003A02807C
:10262000FF00FC0F2C060E082E060E08FFFFFFCF42
:102630000325A14AA300A1499B185A58120F2A4208
:1026400004D05A58120F2A40012A06D10122A24072
:1026500010009B4D2A88104328805A589948024000
:102660008020800510435850B2E7002CBAD1AB59F6
:10267000944A1A4080239B051343AB51B2E7924B17
:102680008D4E1C88002C13D1B023DB00F358002B97
:1026900000DB55E6B2228D4BD200012155E0013D11
:1026A000B3580B40032B08D1002D49D1884C47E685
:1026B000A622864DD2000321F2E7B358002DEED1B9
:1026C000834C3DE60123019A93409BB203937E4BDA
:1026D000039A1B88134210D00221019802F04AFC91
:1026E000019B002B14D1B223DB000121F2580A42D6
:1026F00001D000F04DFF002D1AD1019B0133019351
:10270000744B019A1B683B331B789A42DAD917E65F
:10271000019A019B9032FF32013B92000120B15897
:10272000014201D000F042FF002DE6D0013DF5E767
:10273000013DDAE7C022195892050A431A50DCE736
:102740000023634C0193DBE7013BB058084203D1FF
:10275000002BF9D15E4CF3E5002B08D0B122C02349
:10276000D200B1589B050B43B3500024E8E5584C08
:10277000E6E543331B78002B04D04F4A93695B0096
:102780005B0893610024DBE543334B4A1B785169B6
:10279000002B08D08023DB05194204D0002F04D081
:1027A00091690B4393610024CAE593694A490B4040
:1027B000F8E7380002F026FF0400C1E53E49474A29
:1027C000B8058B58800D9B0A9B0203438B50002455
:1027D000B6E5434A1278002A01D100F0A6FE00981F
:1027E0000838632801D900F0A3FE03F0EBFEE800EF
:1027F000F4000601250131013D014C015801A106FB
:10280000640170017E019601D6011802C0025F03C7
:1028100078039103AA03BE03D703E503F303070478
:102820001B042904370450045F046D047B05A405D0
:10283000CE05FF055406A106A1066D06A106A10658
:10284000A106A106A106A106A106A106A106A10650
:10285000A106A106A106A106A106A106A106A10640
:10286000A106A106A106A106A106A106A106A10630
:10287000A106A106A106A106A106A106A106A10620
:10288000A106A106A106A106A106A106A106A10610
:10289000A106A106A106A106A106A106A106A10600
:1028A000A106A106A106A106A106A106A1067B001C
:1028B0009B00BB00D100C04600002640FC05000084
:1028C0002E060E08FFFFFFCF2C060E0840420F0019
:1028D000FA0F1A0118090E08FFFFFFBF3C050000A0
:1028E00020070E080122C84D6B78E91C01932B7953
:1028F0002E780393FBB22A706A70CB77002B0ED12F
:102900002A71280001F0A6F9041E00D118E56B46D3
:102910001B792E706B706B461B7B2B7110E50023AF
:102920002B71EEE701210022B74D6B78281D019332
:102930002B792E780393FBB229706A70C377022B30
:102940000ED12971280001F085F9041E00D1F7E4A9
:102950006B461B792E706B706B461B7B2B71EFE403
:102960002A71EFE7A84D2B786E1D0193F37F2800A5
:10297000039301232B70F37701F06CF9041E00D14F
:10298000DEE46B461B792B706B461B7BF377D7E439
:102990009D4D2B786E1D0193F37F28000393012337
:1029A0002B700023F37701F055F9041E00D1C7E422
:1029B0006B461B792B706B461B7BF377C0E40023BF
:1029C000914D28006E796B7101F044F9041E00D11D
:1029D000B6E46E71B4E48C4D6B7A28000193002349
:1029E000AE6E6B72AB6601F035F9041E00D1A7E440
:1029F0006B461B79AE666B72A2E4002F01D100F02A
:102A00009AFD3B331B78BB4201D200F097FD0023B7
:102A10007D4D012F0BD1AE7AAB72280001F01AF96F
:102A2000041E00D18CE4012F04D1AE7288E4EE7A4A
:102A3000EB72F2E7EE7283E40123734D2800EE7926
:102A4000EB7101F007F9041E00D179E4EE7177E42F
:102A500000236D4D2800EE79EB7101F0FBF8041EA8
:102A600000D16DE4EE716BE43B0067485A1E934160
:102A7000050055352E782B7001F0ECF8041E00D1BE
:102A80005EE42E705CE401235F48451CEE7FEB772B
:102A900001F0E0F8041E00D152E4EE7750E4002388
:102AA0005948451CEE7FEB7701F0D4F8041E00D1A5
:102AB00046E4EE7744E40123534D28002E7A2B722E
:102AC00001F0C8F8041E00D13AE42E7238E4002365
:102AD0004D4D28002E7A2B7201F0BCF8041E01D156
:102AE000FFF72EFC2E72FFF72BFC4748FBB20500C8
:102AF000013B5A425341002456352E782B70037AFD
:102B0000A34201D1FFF71CFC01F0A4F8041E01D17F
:102B1000FFF716FC2E70FFF713FC052F01D900F00C
:102B200010FD3800384D012303F042FD0316191C37
:102B30001F226E7D6B75280001F08CF8041E01D1F8
:102B4000FFF7FEFB052F01D9FFF7FAFB380003F072
:102B50002FFD1215181B1E21AE7DAB75EBE7EE7D28
:102B6000EB75E8E72E7E2B76E5E76E7E6B76E2E787
:102B7000AE7EAB76DFE76E75FFF7E2FBAE75FFF773
:102B8000DFFBEE75FFF7DCFB2E76FFF7D9FB6E76E9
:102B9000FFF7D6FBAE76FFF7D3FB052F01D900F088
:102BA000D3FC38000023184D03F002FD0316191C56
:102BB0001F226E7D6B75280001F04CF8041E01D1B8
:102BC000FFF7BEFB052F01D9FFF7BAFB380003F072
:102BD000EFFC1215181D2023AE7DAB75EBE7EE7DE3
:102BE000EB75E8E72E7E2B76E5E76E7E6B76E2E707
:102BF000AE7EAB76DFE76E75FFF7A2FBAE75FFF733
:102C00009FFBEE75FFF79CFB30060E082E76FFF754
:102C100097FB6E76FFF794FBAE76FFF791FB386873
:102C2000052801D900F093FCDA4C3B79220003F02F
:102C3000BFFC032E3C4A58662600A532A8361578FC
:102C40001370326818000192627DA634039202F07C
:102C50007FFB2378D049D84003F0BEFC039B306053
:102C60001C1E01D1FFF76CFBCA4E300000F0F2FFD2
:102C7000041E01D1FFF764FB3868052801D9FFF76E
:102C80005FFB330003F094FC4950575E656C2600EF
:102C9000AC32B03615781370326818000192A27DFC
:102CA000AD34039202F054FBD3E72600B432B836B9
:102CB00015781370326818000192E27DB5340392E2
:102CC00002F046FBC5E72600BC32C036157813700B
:102CD000326818000192227EBD34039202F038FB64
:102CE000B7E72600C432C83615781370326818006A
:102CF0000192627EC534039202F02AFBA9E7260006
:102D0000CC32D03615781370326818000192A27E4A
:102D1000CD34039202F01CFB9BE7A5331D70019B91
:102D2000A8363360FFF70CFBAC331D70019BB03647
:102D30003360FFF705FBB4331D70019BB836336079
:102D4000FFF7FEFABC331D70019BC0363360FFF7FE
:102D5000F7FAC4331D70019BC8363360FFF7F0FAF1
:102D6000CC331D70019BD0363360FFF7E9FA386829
:102D7000052801D900F0EEFB864B3A791C0003F0E0
:102D800017FC032E39444F5A1D00A63421782270B7
:102D900001915A7DA8352E680392A533187802F068
:102DA000D7FA23787C49D84003F016FC039B2860AF
:102DB0001C1E01D1FFF7C4FA764D280000F04AFF2F
:102DC000041E01D1FFF7BCFA3868052801D9FFF7C6
:102DD000B7FA2B0003F0ECFB3A424A525A621D004C
:102DE000AD342178227001919A7DB0352E6803921E
:102DF000AC33D3E71D00B534217822700191DA7D20
:102E0000B8352E680392B433C8E71D00BD3421786D
:102E1000227001911A7EC0352E680392BC33BDE743
:102E20001D00C5342178227001915A7EC8352E6864
:102E30000392C433B2E71D00CD3421782270019192
:102E40009A7ED0352E680392CC33A7E76A46127972
:102E5000A633A8351A702E60FFF772FA6A46127907
:102E6000AD33B0351A702E60FFF76AFA6A461279F0
:102E7000B533B8351A702E60FFF762FA6A461279D8
:102E8000BD33C0351A702E60FFF75AFA6A461279C0
:102E9000C533C8351A702E60FFF752FA6A461279A8
:102EA000CD33D0351A702E60FFF74AFA394D2E0017
:102EB000AB7CA2360193337828000393012337704B
:102EC000AB7400F0C7FE041E01D1FFF739FA6B4660
:102ED0001B7B33706B461B79AB74FFF731FA2D4DBA
:102EE0002E00A336337828000193EB7C37700393D0
:102EF0000123EB7400F0AEFE041E01D1FFF720FAAF
:102F00006B461B7933706B461B7BEB74FFF718FA2B
:102F1000204D2E002B7FD636019333782800039363
:102F2000012337702B7700F095FE041E01D1FFF7C7
:102F300007FA6B461B7B33706B461B792B77FFF7C9
:102F4000FFF9144800240500D8352E882F80837F90
:102F5000A34201D1FFF7F4F900F07CFE041E01D179
:102F6000FFF7EEF92E80FFF7EBF90A480024050081
:102F7000DA352E782F70837FA34201D1FFF7E0F975
:102F800000F068FE041E01D1FFF7DAF92E70FFF79A
:102F9000D7F9C04630060E0840420F000123CF4D3E
:102FA0002800AE7FAB7700F055FE041E01D1FFF77D
:102FB000C7F9AE77FFF7C4F90023C84D2800AE7FEC
:102FC000AB7700F047FE041E01D1FFF7B9F9AE77E9
:102FD000FFF7B6F9C14800240500D4352E782F70CC
:102FE000C37EA34201D1FFF7ABF900F033FE041E0C
:102FF00001D1FFF7A5F92E70FFF7A2F9B748002419
:103000000500D5352E782F70C37EA34201D1FFF77E
:1030100097F900F01FFE041E01D1FFF791F92E7001
:10302000FFF78EF90123AD4D2800EE7EEB7600F020
:1030300011FE041E01D1FFF783F9EE76FFF780F948
:103040000023A64D2800EE7EEB7600F003FE041E62
:1030500001D1FFF775F9EE76FFF772F99F4D2E005B
:103060006B7FD736019333782800039301233770A1
:103070006B7700F0EFFD041E01D1FFF761F96B469D
:103080001B7B33706B461B796B77FFF759F9934BBA
:103090005C79002C00D060E23A689A627A68DA6261
:1030A000BA681A63FA685A63FFF74AF901238B4D2D
:1030B00028006E796B7100F0CDFD041E01D1FFF781
:1030C0003FF96E71FFF73CF93868052800D947E2EF
:1030D000824B03F06DFA031B222930371A000121BD
:1030E00096321E7B15881973B9881800118000F07C
:1030F000B1FD041E38682CD1052801D9FFF720F94D
:10310000764D03F055FA4D6A89A9BFD51A00012101
:1031100098325E7B15885973E6E71A0001219A32CE
:103120009E7B15889973DFE71A0001219C32DE7BB4
:103130001588D973D8E71A0001219E321E7C1588A4
:103140001974D1E71A000121A0325E7C15885974E8
:10315000CAE7052800D906E2604B03F029FA030804
:103160000D12171C1E7396331D80FFF7E9F85E736E
:1031700098331D80FFF7E4F89E739A331D80FFF7A4
:10318000DFF8DE739C331D80FFF7DAF81E749E3380
:103190001D80FFF7D5F85E74A0331D80FFF7D0F8CF
:1031A0006B7A002B03D0280000F0A0FCA8662B004F
:1031B000A5331878002801D0FFF7C2F802F0C8F84C
:1031C0002B00A6331B784649A83599404B081818A0
:1031D00003F002FA2860FFF7B3F8AB7A002B05D0B2
:1031E0002900012000F0A0FC2B1DD8672B00A5337F
:1031F0001878012801D0FFF7A3F802F0A9F82B00F6
:10320000A6331B783649A83599404B08181803F0A7
:10321000E3F92860FFF794F8EB7A002B06D0290039
:10322000022000F081FC2B008C3318602B00A533AA
:103230001878022801D0FFF783F802F089F82B00F4
:10324000A6331B782649A83599404B08181803F077
:10325000C3F92860FFF774F82B00A533187803280A
:1032600001D0FFF76DF802F073F82B00A6331B783E
:103270001B49A83599404B08181803F0ADF9286090
:10328000FFF75EF82B00A5331878042801D0FFF76C
:1032900057F802F05DF82B00A6331B781049A835CB
:1032A00099404B08181803F097F92860FFF748F881
:1032B0002B00A5331878052801D0FFF741F802F05C
:1032C00047F82B00A6331B780549A83599404B08D1
:1032D000181803F081F92860FFF732F830060E085D
:1032E00040420F003A68BC4B0024DA661A00B988E5
:1032F000703211801A00B979723211701A00F9799E
:10330000733211701A003989743211801A00B97A37
:10331000763211701A00F97A773211701A00B98971
:10332000783211801A00B97B7A3211703A8A7C3374
:103330001A80FFF705F8A84D6E7A002E00D015E12F
:10334000012328006B7200F0D1FBA866280000F072
:1033500081FC041E03D0AE666E72FEF7F1FF2B00F7
:10336000A5331B78002B01D0FEF7EAFF01F0F0FF38
:103370002B00A6331B789949A83599404B0818189B
:1033800003F02AF92860FEF7DBFF3A68002A00D133
:10339000EFE03B331B789A4200D9EDE07B681E7862
:1033A0005D789C78D87819798B4B012A10D11A0056
:1033B000843216701A00853215701A008632147025
:1033C0001A0087321070883319700024FEF7B8FF96
:1033D0001A00903216701A00913215701A0092324B
:1033E00014701A00933210709433EDE7012F06D158
:1033F000794A927A002A09D0794CFEF7A1FF022F70
:1034000004D1754AD27A002A00D0B8E03B331B7849
:10341000BB4200D2B6E0002F00D1B6E06E4D2900CD
:10342000012F12D1380000F07FFB2B1DD867AF723F
:10343000280000F00FFC041E16D00023012F0DD130
:103440002A1DD367AB72FEF77BFF022000F06CFBF6
:103450002B008C3318600123EB72E9E72A008C32D1
:103460001360EB72FEF76CFF2B00A5331878431E38
:10347000012B01D9FEF764FF01F06AFF2B00A63390
:103480001B785649A83599404B08181803F0A4F842
:103490002860FEF755FF504D2E002B7DA43601937A
:1034A000337828000393012337702B7500F0D2FB8B
:1034B000041E01D1FEF744FF6B461B7B33706B4645
:1034C0001B792B75FEF73CFF0122434B00249A71B8
:1034D0009F64FEF735FF0024FEF732FF414CFEF7F4
:1034E0002FFF404CFEF72CFF3E4CFEF729FF3D4CD2
:1034F000FEF726FF3B4CFEF723FF3A4CFEF720FF7A
:10350000384CFEF71DFF374CFEF71AFF354CFEF71F
:1035100017FF344CFEF714FF334CFEF711FF334C0A
:10352000FEF70EFF314CFEF70BFF2E4CFEF708FFA7
:103530002C4CFEF705FF2E4CFEF702FF2C4CFEF73D
:10354000FFFE284CFEF7FCFE264CFEF7F9FE254C4C
:10355000FEF7F6FE234CFEF7F3FE264CFEF7F0FED8
:10356000204CFEF7EDFE1F4CFEF7EAFE224CFEF764
:10357000E7FE1F4CFEF7E4FE1D4CFEF7E1FE184C83
:10358000FEF7DEFE164CFEF7DBFE154CFEF7D8FE0E
:10359000002D01D1FFF7B1F8B122C023D200B158FC
:1035A0009B050B43B3500024FFF7A7F8002D01D172
:1035B000FFF7A3F8C020114A9B001488039AC000AB
:1035C00014400F4A9B18002C01D1FFF7B3F81A588A
:1035D0000C490A401A50E6E730060E0840420F0038
:1035E0002D0F1A01FF0F1A01F90F1A01FE0F1A0110
:1035F000BD0F1A01590F1A013E0F1A012E060E08AF
:1036000000002640FFFFFFCF73B520220020344B7F
:10361000D100591A0531FF31013A0860002AF7D16B
:1036200030491960304999603049196130499961D0
:1036300030491962304999623049196330499963B8
:10364000304919643049096808003C300078042882
:1036500000D92E4A9A640022052800D92C4A1A65FE
:103660004A6801241000083098652A4864421866A8
:103670002948DC6758662948986629481867294808
:1036800012189A6700221500981806000832803632
:10369000843035600460802AF6D185220B6A52019D
:1036A0009B18802252039A6004236A4613808B8EF3
:1036B000684605331C495380019502F02FF8002815
:1036C00000D001BE6B4600229B5E002B06DB1F2252
:1036D00013401E3A9A401300144A136073BDC0464B
:1036E0001C090E0808002640000726400407264053
:1036F00008072640100726408403264088032640FA
:103700008C0326409003264018090E089403264097
:10371000980326400400264000FF03F04805264099
:103720004405264060F00000F922001000E100E0AE
:10373000064A0300126800203C3212789A4204D9EB
:10374000E033034A9B009858C00F704718090E08D1
:103750000000264070B50F4B1B683B331A78431EA0
:10376000591E8B419A4213D90B4B0C4D8000C41843
:1037700063590B4A01201A4080239B051343635170
:1037800002F030F8002063595B005B08635170BDA4
:103790000448FCE718090E0800002640FC0500005C
:1037A000FFFFFFCF01004A00094B1B683C331B7829
:1037B00083420AD9E022074B8000C0189200835848
:1037C0005B005B088350002070470348FCE7C0465D
:1037D00018090E080000264001004A0010B50B4BE6
:1037E0001B683C331B7883420DD90F290BD8E0228C
:1037F0000F24074B8000C01892008358A34319433D
:103800008150002010BD0348FCE7C04618090E088F
:103810000000264001004A00022817D006D80028E0
:1038200027D0012810D0022040420CE01223FF33A1
:1038300098420DD01423FF3398420CD0033B98429A
:10384000F1D1FA20C0017047886CFCE7886AFAE77A
:1038500080200002F7E7084B1B683D3318780138D9
:10386000431E9841054B4042184080231B02C0185C
:10387000E9E70348E7E7C04618090E08FE7FFFFFA7
:1038800000127A0002235B4210B51360314B140022
:103890001B681A003A321278824258D9052856D845
:1038A00002F086FE03192E43494F0B7B002B4ED0AE
:1038B0004B7A002B08D00B007A331B78022B03D0F5
:1038C0008B6E2360002010BD0B0096331888FFF725
:1038D000A3FF2060F6E74A7B002A38D03B331B78F1
:1038E000002B0AD08B7A002B07D00B0088331B7873
:1038F000022B02D00431CB6FE3E70B009833E5E7EE
:103900008A7B002A23D03B331B78012B0AD9CB7A40
:10391000002B07D00B0094331B78022B02D08C3184
:103920000B68CEE70B009A33D0E7CB7B002B0ED091
:103930000B009C33CAE70B7C002B08D00B009E3396
:10394000C4E74B7C002B02D00B00A033BEE702483B
:10395000B9E7C04618090E08FE0F1A01032819D04E
:1039600004D801280FD028D948790DE01223FF335D
:10397000984214D01423FF33984212D0033B98424C
:103980000BD00F4805E08879434258410C4B404228
:10399000184070470231C87FF6E7C879F4E7087A23
:1039A000F2E70131CB7F002BEBD0064B1B683D3398
:1039B00018780138431E9841E8E70020E9E7C0463F
:1039C000FE0F1A0118090E0810B51B4B1B683A337D
:1039D0001B7883422DD905282BD802F0E9FD030C72
:1039E00012181E240B7B002B23D00B009633188853
:1039F000FFF7B4FF10BD4B7B002B1AD00B009833A0
:103A0000F5E78B7B002B14D00B009A33EFE7CB7BD1
:103A1000002B0ED00B009C33E9E70B7C002B08D069
:103A20000B009E33E3E74B7C002B02D00B00A0334E
:103A3000DDE70248DEE7C04618090E08FE0F1A014E
:103A40000300A8331B6810B50400002B02D00848FF
:103A5000584310BD0300A533187801F079FC02002B
:103A60000120A6342378984040088018D840F0E719
:103A700040420F0010B5040001F0F4FB002801D013
:103A8000044810BD0449200001F0C8FC0028F8D00B
:103A9000F6E7C046FD0F1A011027000070B50500BB
:103AA0001400FFF79BFE002818D10D4B1B683C3318
:103AB0001B789D4212D2032C10D8E021AB00302598
:103AC000084A89009B185A582401AA4322435A5095
:103AD00080225C58120622435A5070BD0248FCE70F
:103AE00018090E0800002640FD0F1A01030010B54A
:103AF0000400963318882100FFF78EFE0300002093
:103B00009A1C0FD022007032118881420AD0E06ED8
:103B10007334584302F060FD21784B1E9941013106
:103B200002F05AFD10BD000070B500250C00A8423F
:103B300021D01B4B1B683B331B7883421BD30128CE
:103B40001BD10B0098331888FFF766FE2300220074
:103B5000843385321B78117886342578821C1BD0FB
:103B600000291BD0002D06D0584302F035FD290056
:103B700002F032FD0500280070BD0228FBD10B00C9
:103B80009A331888FFF748FE2300220090339132C1
:103B90001B7811789234E0E70025ECE70D00EAE7A6
:103BA00018090E08F8B504000F00012932D10300EE
:103BB000817A427B04309833C66F83301B88057846
:103BC0000020814225D0824231D018002100FFF729
:103BD00023FE184BC018184B984228D86B1E9D41E5
:103BE000164B6D421D40164BED182379002B1AD051
:103BF000AE421CD3134B9E4219D821003800FFF768
:103C000093FF301A464270410F4E40420F4B3040F6
:103C1000C018F8BD0300C17A827B9A338C301B88B0
:103C20000668C579CCE7AE4201D3094BE3E7074804
:103C3000EFE7C04600F7C2FF00879303C863E3FFC6
:103C400020BCBE0080F0FA0202F0E5FEFE0F1A0171
:103C500080D1F008F0B504008FB0002801D100F049
:103C6000DEFFA621C44BC9005A58D24392071ED08A
:103C70005B584379002B1AD0C04A836A9B18C04A0C
:103C8000934201D900F0CEFFC36A013B632B01D9F7
:103C900000F0C8FF036BBB4A013B934201D900F01F
:103CA000C1FF436B013B934201D900F0BBFFA379F5
:103CB000002B0ED02279A36C002A00D105E1B24A74
:103CC000934201D900F0B1FFE36C002B01D100F069
:103CD000ACFF237B0293002B0FD0AC4B1B683A3315
:103CE0001B78002B09D02300963318882100FFF79A
:103CF00035FE002801D000F09BFF637B0393002B6F
:103D00000FD0A24B1B683A331B78012B09D9230033
:103D1000983318882100FFF721FE002801D000F019
:103D20008AFFA37B0493002B0FD0984B1B683A3378
:103D30001B78022B09D923009A3318882100FFF73A
:103D40000DFE002801D000F079FFE37B0593002BE6
:103D50000FD08E4B1B683A331B78032B09D92300F5
:103D60009C3318882100FFF7F9FD002801D000F0EE
:103D700068FF237C0693002B0FD0844B1B683A33DB
:103D80001B78042B09D923009E3318882100FFF7E4
:103D9000E5FD002801D000F057FF637C0793002B5E
:103DA0000FD07A4B1B683A331B78052B09D92300B7
:103DB000A03318882100FFF7D1FD002801D000F0C2
:103DC00046FFB0236C4ADB00D358002B5CDB637AE0
:103DD000002B59D0029B002B01D100F03BFF2300A8
:103DE000963318882100FFF717FD694BC018694BFF
:103DF000984201D900F02EFF674AA36E9B182279E2
:103E0000002A64D0654A934201D900F023FFE36E93
:103E1000634A013B934201D900F01CFF2300703339
:103E20001B88604A013B9BB2934201D900F012FF0C
:103E3000230072331B78042B01D900F00BFF230001
:103E40007433594A1B88934201D900F003FF2300C1
:103E500076331B780F2B01D900F0FCFE230077335B
:103E60001B780F2B01D900F0F5FE230078334F4962
:103E70001B888B4201D900F0EDFE23007C331B88A8
:103E8000934201D900F0E6FE404B1D682B003B3306
:103E90001E78002E01D100F0FFFEA37A002B0DD07A
:103EA000C023354ADB00D358002B07DB012120005B
:103EB000FFF778FE002801D000F0D5FE0027012E84
:103EC00001D900F0D5FE00F0E7FE394AF8E6394A9C
:103ED00099E7002F01D100F0DFFE38000FB0F0BDF0
:103EE000E379002B01D100F0EBFE637D002B3AD08B
:103EF0002B003C331B78002B35D02300A5331E78D4
:103F000021003000FFF760FD00282CD13A352B78D6
:103F10009E4228D2052E26D8300002F049FB1226F8
:103F200051575D63237ADCE7631CDB7F002B01D1F3
:103F300000F0C6FE2B003D331B78012BD5D000F0DE
:103F4000BFFE029B002B0ED0230096331B88002B54
:103F500009D109AA21003000FFF794FC164B099AF9
:103F600007009A4244D8154FB7E7039B002BFAD0BD
:103F700023009833EAE7C0460000264000DC0BFF30
:103F8000C0EA2101E703000080F0FA0218090E08D8
:103F900018FCFFFF18DDF50500CA91FE80BA8C0100
:103FA000FEFF0300FE1F0000FF010000FF1F0000D6
:103FB00000E1F50500AB87043F0D03009F0F1A01D8
:103FC000049B002BCFD023009A33BFE7059B002B27
:103FD000C9D023009C33B9E7069B002BC3D0230034
:103FE0009E33B3E7079B002BBDD02300A033ADE782
:103FF000002FB8D12300A8331B68002BB3D0B54ED7
:10400000B54D7343AB42AED82300A6331B78032BC8
:10401000A9D8A37D002B1DD0B04B1B683C331B7867
:10402000012B17D92300AC3318782100FFF7CCFC03
:10403000002801D000F09FFC2300AD331A78033331
:104040001B687343AB4201D900F095FC032A01D9E8
:1040500000F091FCE37D002B1DD0A04B1B683C338E
:104060001B78022B17D92300B43318782100FFF7EF
:10407000ABFC002801D000F0A9FC2300B5331A786E
:1040800003331B687343AB4201D900F09FFC032A42
:1040900001D900F09BFC237E002B1DD08F4B1B68A9
:1040A0003C331B78032B17D92300BC33187821002D
:1040B000FFF78AFC002801D000F080FC2300BD330C
:1040C0001A7803331B687343AB4201D900F076FCC6
:1040D000032A01D900F072FC637E002B1DD07F4BB8
:1040E0001B683C331B78042B17D92300C433187882
:1040F0002100FFF769FC002801D000F07CFC2300C0
:10410000C5331A7803331B687343AB4201D900F0FF
:1041100072FC032A01D900F06EFCA37E002B1ED096
:104120006E4B1B683C331B78052B18D92300CC330E
:1041300018782100FFF748FC002801D000F09BFC14
:1041400022002300D0321268CD3356431B78AE4292
:1041500001D900F090FC032B01D900F08CFCE37E28
:10416000002B0AD1637F002B26D1A37C002B49D1E1
:10417000E37C002B58D15A4FAFE62300D4331B7891
:10418000210018000293FFF71FFC002812D126001F
:10419000D5363378042B0DD809AA21000298FFF7F1
:1041A00071FB002806D13378099ADA4013004D4A92
:1041B0009342D7D94C4F90E62300D7331B78002B7E
:1041C00003D0012B05D0494F87E6237A002BCCD1B1
:1041D000F9E7237F002BF6D02300D6331B78012B81
:1041E000F3D0002B0CD0032BEDD1631CDB7F002B15
:1041F000E9D03A4B1B683D331B78012BE3D1B4E780
:10420000E379E3E7637D002B01D1394F65E62000B8
:10421000FFF716FC2300A2331978013102F0DCF914
:10422000304B9842A4D9F0E7637D002BA3D0200047
:10423000FFF706FCA8429ED82300A3330393197806
:10424000013102F0C9F92379002B0AD0294B984299
:1042500091D8A37F002B06D1237D002B58D1264F68
:104260003BE6264BF3E723000222D8331B88FF32BC
:10427000934204D022D8002B28D0012B24D1617D79
:10428000002921D00226934208D01D4AB619934234
:1042900004D01C4A0436934200D0073E2000FFF7AA
:1042A000CFFB2300DA331978013102F095F93100A0
:1042B00002F092F90B4B9842CED905E010498B429F
:1042C000DDD010498B42DAD00F4F06E601260F48A9
:1042D000E7E7C04640420F0080D1F00818090E08F9
:1042E0008C0F1A010084D7178F0F1A018E0F1A0135
:1042F0008D0F1A0140787D018B0F1A0100E1F50541
:104300000102000001030000890F1A0100127A0067
:10431000E37C002BA3D02000FFF792FBA84200D93A
:1043200029E7039BE61C1978251D013102F054F999
:104330002300A43305931978013102F04DF9C74BDE
:1043400098428CD89621002001F090FA2378002B17
:1043500033D06378002B0FD0F07F012806D9631D7E
:10436000DB7F002B10D101F05BFC0FE001F0C0FD02
:104370000028F4D0BA4FB0E5E87F022801D0052824
:10438000EDD101F00DFEF3E701F026FC0028F1D19C
:10439000B44BB5495A6CFF200A40E82189010A4311
:1043A0005A64A278002A79D05A6C120A02403A2A3A
:1043B00003D1596CAD4A0A435A64AD4B1B683D3377
:1043C0001B780293012B0CD1AA4EAB4D631C725982
:1043D000DB7F92006DD5002B03D17359DB00DB0826
:1043E000735108269F4A237A15680292354071D08E
:1043F000002B07D17B2001F0F5F9029B029A1B6884
:10440000B3431360237F9B4E002B1AD02300A022BE
:104410000325D6331B78D20004930499B3582B405C
:1044200099420ED001F092FF002801D000F018FC54
:10443000A0220499D200B3582940AB430D001D437C
:10444000B550A621C90073586279DB439B0700D1A0
:1044500082E07358002A00D185E001F0C7FFA06B0D
:10446000002810D0E36B002B0DD00025216C2B0011
:104470002A000095FDF772FC00952B002A00616C64
:10448000E06BFDF76BFC636B226BE16AA06A00F0E6
:1044900097FC002800D1C0E0784F1EE55A6C120A44
:1044A00002403A2A89D15A6C754802401143596436
:1044B00083E7002B95D001F099FF802372591B06EA
:1044C00013437351029801F073F9C0237259DB054D
:1044D000134385E7002B95D001F088FFA06D0028DD
:1044E0000FD0E36D002B0CD02B002A00216E00951D
:1044F000FDF734FC00952B002A00616EE06DFDF79E
:104500002DFC230056331B785E4A002B17D0029BEC
:104510001B681A4080235B021343029A042613602F
:10452000029B594D1A6808231343029A1360029B99
:104530001B6933420CD1002D05D1544FCDE4029BB1
:104540001B681340E9E7012001F04CF9013DEEE75B
:10455000002D00D056E7F0E7002A04D14C4AB358AA
:104560005B005B08B350A379002B0ED0E06C0028F1
:1045700008D0230054331B7808220093216D0023B8
:10458000FDF7ECFBA06C00F011FCA37C002B0FD01E
:10459000374B35481B68190008311A68CB6FD218A1
:1045A0002300A23311681B7801401B020B431360E8
:1045B000E37C002B0DD02E4B1B681A1D1968D36F9E
:1045C000C918039B0A681B7812021B06120A1343C0
:1045D0000B60237D002B0DD0254B23481B68191D34
:1045E0001A68CB6FD218059B11681B7801401B021B
:1045F0000B4313602500122296352B88FF3293421D
:1046000023D12300A533197800291ED1012000F001
:10461000B1FC002807D01F4F5FE41F4800F06EFC7C
:104620000028A0D038E70121FFF7D8F800280AD1E8
:10463000237B002B36D02988002000F09BFC00282B
:1046400030D0164F49E4164F47E4230098331988B9
:10465000012000F08FFC0028EAD0DCE700E1F5053E
:104660006F0F1A0100002740FF00FFFF003A0020F3
:1046700018090E08000026403C0500005F0F1A01D3
:10468000FFC5FFDFFFFFFEFF40420F005A0F1A0178
:104690002C0500004E0F1A01B80B00004F0F1A0135
:1046A0000F0F1A01A37B002B0AD023009A3319881D
:1046B000022000F05FFC002802D0D04FFFF70DFC75
:1046C000E37B002B67D1237C002B75D1637C002B0F
:1046D00000D083E0B022D200B158637A002900DB19
:1046E0008FE0002B11D1B120C0003358C4491940CC
:1046F00080239B050B433350B3585B005B08B350DA
:10470000C04AB3585B005B08B3502300A533039342
:1047100019780020FFF762F8002894D1BA4B1B6883
:104720003C331B78002B8ED02300A6331A78032A43
:1047300089D8E02189007358303012018343134334
:10474000122273502B88FF32934200D192E0AE4D7B
:104750002B683B331B78002B00D09EE00120FEF736
:10476000E7FFA37D002800D108E1002B00D1FCE089
:104770000220FEF7DDFFE37D002800D00AE1002BD8
:1047800000D109E12300B5331A78013B19780220E2
:10479000FFF784F918E19C4B1B683A331B78032B15
:1047A00091D923009C331988032000F0E3FB0028F3
:1047B00089D0964FFFF791FB934B1B683A331B78D8
:1047C000042B83D923009E331988042000F0D2FBE8
:1047D000002800D17AE78E4FFFF77FFB8A4B1B68DA
:1047E0003A331B78052B00D874E72300A0331988CF
:1047F000052000F0BFFB002800D16BE7854FFFF7D5
:104800006CFB002B00D180E701F0F0FDE36E09A8FE
:104810000993230070331B888380230072331B7835
:104820008371230073331B78C371230074331B8897
:104830000381230076331B788372230077331B7840
:10484000C372230078331B88838123007A331B785B
:10485000837323007C331B88038200F005FC00284F
:1048600005D16D4800F08AFC002800D14DE76B4F60
:10487000FFF733FB039B1B78002B00D067E7637BBC
:10488000002B00D1C7E6230098331988012000F0DF
:1048900071FB002800D15AE7BDE6C023DB00F258C7
:1048A000A37A002A0BDA002B27D101F09FFD01200B
:1048B000FEF750FF002820D0594FFFF70EFB002BCA
:1048C0001BD0230084331B7806AA1373230085337F
:1048D0001B785373230086331B789373230087332D
:1048E0001B78D373230088331B78137401F07EFD8B
:1048F00009A90120FFF7BEF8DCE72B683B331B78E2
:10490000012B00D82AE7474BF258E37A002A0DDA48
:10491000002B00D022E701F069FD0220FEF71AFF0C
:10492000002800D11AE7404FFFF7D7FA002B00D13B
:1049300014E7230090331B7806AA137323009133E6
:104940001B785373230092331B78937323009333A4
:104950001B78D373230094331B78137401F046FD46
:1049600009A90220FFF786F8DAE70120FEF71CFF0D
:10497000002800D1FCE62D4FFFF7AFFA002B00D145
:10498000F6E62300AD331A78013B19780120FFF7D2
:1049900085F8EDE7002B14D02B683C331B78032BF4
:1049A00017D90320FEF7C4FE237E002846D0002B33
:1049B0000FD10320FEF7F8FE00280AD01C4FFFF7A6
:1049C0008CFA0220FEF7F0FE0028E5D0194FFFF721
:1049D00084FA2B683C331B78042B3AD90420FEF769
:1049E000A7FE637E002849D0002B32D10420FEF7B9
:1049F000DBFE00282DD0104FFFF76FFA4D0F1A0184
:104A0000FFFFFFCF8C05000018090E084C0F1A019C
:104A10004B0F1A014A0F1A01400D03003F0F1A01F4
:104A20002F0F1A01040600002E0F1A019E0F1A0103
:104A30009C0F1A019D0F1A019B0F1A01002BC8D061
:104A40002300BD331A78013B19780320FFF726F8BD
:104A5000B2E72B683C331B78052B1AD90520FEF7EB
:104A600067FEA37E00284CD0002B12D10520FEF754
:104A70009BFE00280DD0944FFFF72FFA002BE8D0B3
:104A80002300C5331A78013B19780420FFF706F894
:104A9000AFE78E4BA27FF15800293DDA002A03D1FF
:104AA000F25852005208F250A0238021DB00F05847
:104AB0000902E27E08424DD0002A03D1F25884490F
:104AC0000A40F250637F002B0DD0029BC0211A6870
:104AD0002300D7331B7889001B020B407D490A4015
:104AE0001343029A1360230055331D787A4B1B78C9
:104AF000AB425BD001F02AFC00284FD0774FFFF784
:104B0000ECF9002BC5D02300CD331A78013B19787E
:104B10000520FEF7C3FFACE7002AC5D02100220024
:104B2000DA310878F158D832490049081288F15032
:104B3000F5586B49000429406A4D2A400A43F25057
:104B4000F25869490A400243F2508022F158120695
:104B50000A43A8E7002AB5D020002200D53000780B
:104B6000D432127884465A4DF05828401502F0226B
:104B7000F0501201F0582A405C4D28400243E025D5
:104B80006046F2500003ED01F258054058480240DB
:104B90002A43F250F2581143F15093E70121554A4C
:104BA000B3588B432B43B3504B4B1D70514DE3799E
:104BB0007259002A24DA002B12D1A32000F012FE31
:104BC0007359002B0CDA01F0C1FB002896D1C023E9
:104BD0005B00F358DB0791D473595B005B0873519A
:104BE0002378002B08D0637D002B05D02300A83349
:104BF0002079196800F03AFE01F0F8FBFFF76DF933
:104C0000002BEDD07359002BEADB01F09FFB00284D
:104C100000D073E7802372591B061343DFE7364F3A
:104C2000FFF75BF9354FFFF758F9354FFFF755F9A7
:104C3000344FFFF752F9344FFFF74FF9334FFFF777
:104C40004CF9334FFFF749F9324FFFF746F9324F2E
:104C5000FFF743F9314FFFF740F9314FFFF73DF9C7
:104C6000304FFFF73AF9304F012E01D8FFF735F9F1
:104C7000E37A002B01D1FFF72CF9002F01D0FFF7C9
:104C80002CF92A4B2A4AD358002B05DB022120009D
:104C9000FEF788FF0028E0D1237F002B01D1FFF72A
:104CA00024F92300D6331B78012B01D1FFF73AF901
:104CB000002B01D1FFF714F9032B01D1FFF734F9D1
:104CC0001C4FFFF70AF9C0469A0F1A0104050000AD
:104CD000FF7FFFFFFFFCFFFF21070E085C0F1A019B
:104CE000FEFCFFFF01030000FFFF00FFFFF0FFFFDE
:104CF000FF8FFFFF0C050000FE0F1A01EF0F1A01D6
:104D0000EE0F1A01DF0F1A01DE0F1A01DD0F1A0173
:104D1000DC0F1A01DB0F1A01DA0F1A01CF0F1A018B
:104D2000BE0F1A011F0F1A01BF0F1A01040600005F
:104D300000002640AF0F1A0170477047F0230A04A5
:104D40001B0330B51A400F240B0023401A43084BB5
:104D50001D68830228691B188020C0011A5018584A
:104D60002040401A411E884102494042084030BD5F
:104D700018090E080300C200044B10301B688002A3
:104D80001B69C0580F2318407047C04618090E0809
:104D9000A6220549D2008B580220DB439B0702D094
:104DA000012388581840704700002640024B984263
:104DB00001D8024B1860704700E1F5052C070E087A
:104DC000F0B516001F003B4A3B4B0C00D15885B094
:104DD000029001920393002967DB3849384A43184F
:104DE000934264D8631E632B61D8364A731E934284
:104DF0005DD8354A7B1E934259D8FA21F530890097
:104E0000FF3001F0E9FB05003048310047437008EE
:104E1000381801F0E1FB80228446102300201202A2
:104E2000010011430F004F43BC4500D30800013B74
:104E30005208002BF4D12900254B614358434B08FD
:104E4000C01801F0C9FB234B984230D96D43224B67
:104E50002249E81801F0C0FB64436043642132300A
:104E600001F0BAFB1E49704301F0B6FB03281ED8BF
:104E7000012801D8012358401A4A019B1A499B581E
:104E800000031940194B0B431843019B0399985099
:104E9000019B039A00209A5802231343019A53500E
:104EA000134B029A1A6005B0F0BD1248FBE7124896
:104EB000F9E7C046000026402C05000000DC0BFF8F
:104EC000C0EA2101E7030000CF07000080841E0034
:104ED000B36D0200890200005DF70000BBEE010027
:104EE000A0BB0D0020FF000008C0FFFFF70300007B
:104EF00030070E0803004A0001004A00124A134B13
:104F000070B5D158050000291BDB80212C00D0583A
:104F100009060143D150FFF73BFF022801D0002CC6
:104F20000AD10020854206D0601E8441084B6042B1
:104F30001840084BC01870BD012000F053FC013C24
:104F4000E9E70548F7E7C046000026402C050000C9
:104F5000FEFFB5FF02004A0003004A0010B5FFF74C
:104F600017FF0023022801D1014B1B68180010BD58
:104F700030070E08104B1B683A331B78834219D94F
:104F8000042910D94B1EFF3B132B13D81F231940A4
:104F90000A4B8000C018C02304229B00C15040333C
:104FA000C250002070470723D0301940034B8000C7
:104FB000C150F6E70248F5E718090E080000264040
:104FC00001004A00094A83009B18D0229200985899
:104FD00007221040042807D1C022920098581F23AE
:104FE00003408020400018437047C0460000264020
:104FF00010B5FFF7E7FF02281CD005D8002814D011
:10500000012814D0002011E01223FF33984214D05D
:105010001423FF33984218D0033B9842F2D10C4A34
:105020000C4BD058C00FC00300E00B4810BD0B4B19
:105030001868FBE7FFF792FFF8E7094B18690423AC
:105040001840F3D080200002F0E7014A054BE8E762
:10505000000026400C05000000127A002C070E0804
:10506000000027403C05000070B5B024224AE4004F
:105070001359002B3DDBC17903684D1EA9419B03E9
:1050800009069B0B0B431351038984881B491B049E
:10509000E4040B40E40C2343194C1A4D1351FF2434
:1050A000C37AE0261B0123408489F60024022C40A9
:1050B0000F252343847A2C40C0252343847BAD05F0
:1050C00024072C402343B124E400135183790E4C70
:1050D0001B02155933400D4E35402B431351038AA3
:1050E00000201B0415590B40094929400B4313515B
:1050F00070BD0848FCE7C046000026400000FF01E4
:105100008405000000FF1F008C050000FFF8FFFF72
:10511000FFFF00FE03004A00B023154ADB00D3580E
:1051200010B59903DB01DB0F890BC371114B0160D3
:10513000D3580F24D904DB01DB0D0381B123DB003D
:10514000D358C90C8180190021408172190921406E
:10515000C172D9029B009B0F8373074BC90CD358B4
:1051600081815A05DB01520FDB0D8271038210BD74
:1051700000002640840500008C050000F7B5802261
:10518000B22607000500324B324C1206E158F600F9
:105190000A43E25000930422A359134201D1002D87
:1051A00035D1B1208023C00022582B499B050A40ED
:1051B000134323500191002F01D0002D06D0B022BF
:1051C0008023D200A1581B060B43A3500126B22313
:1051D000DB00E358334224D1002D1DD1002F24D011
:1051E000B121C9006258019B1C481A4080239B05CD
:1051F0001343B0226350D200A3585B005B08A35056
:10520000009B009AE3585B005B08A350FEBD0120A1
:1052100000F0E8FA013DBEE7300000F0E3FA013D9E
:10522000D5E7002F01D0002DDAD0B122C023002015
:10523000D200A1589B050B43A3508742E6D0681EBD
:1052400085416842064D054B2840C018DEE7C04640
:105250008C05000000002640FFFFFFCF02004A003F
:10526000FEFFB5FFF0B5204B1B683B331B78834234
:1052700033D31E4B80001E4CC0180359002B2ADB71
:105280008E78B31E0E2B28D84F787B1E112B24D876
:105290000B78CD789C46002D21D1152B1DD970237C
:1052A0009C451AD80A79022A0AD07F236146194000
:1052B0000B003F023B4336043343ED062B430351BF
:1052C000C0211207890503590A400A490B401A43B5
:1052D00002510020F0BD0848FCE70848FAE7122B0D
:1052E000FBD93823DCE7C04618090E080000264029
:1052F000FC050000FFFFFFCF03004A0001004A0049
:1053000010B5104B421E1B683B331B78934216D9D5
:105310007F221F248030FF300B4B8000C3581A407F
:105320000A701A0C2240180A8A701A012040E240C2
:10533000487000209B009B0FCA700B7110BD034882
:10534000FCE7C04618090E080000264001004A008C
:10535000F0B587B00400FFF74BFE0600002C38D1F3
:1053600001AD14222100280001F02BFB2800FFF7DB
:10537000D3FEB023274ADB00D358002B03DAAC7BE3
:10538000023C631E9C41EA79019F531E9A41A88802
:105390000132002C1AD0002818D0002A16D0002381
:1053A000190001F0C5F900230C0005003A00300097
:1053B000190001F0BDF9E6076A0832436308801856
:1053C00059412A00230001F093F90600300007B08C
:1053D000F0BD114B1B683B331B78A342F6D301ADE4
:1053E00005220021280001F0ECFA20002900803479
:1053F000FFF786FFFF34074BA400E3580024A342C5
:1054000003DA2C79023C631E9C412F786878AA78D5
:10541000BFE7C0460000264018090E08F8B5174B34
:105420000D001B683B331A78431E9A4223D9144B54
:105430008000C41880232E000127124A1B06A158A1
:105440000B43A350104BE3583B420AD1002E03D12B
:1054500068426841404209E0380000F0C3F9013E6B
:10546000F0E7281E08D0701E86417042074B184096
:10547000074BC01800E00748F8BDC04618090E08E1
:1054800000002640FC0500003C060000FEFFB5FFC2
:1054900002004A0001004A00F7B5484B0091150090
:1054A000984200D987E09A4200D984E0444B99425F
:1054B00000D980E00122434B1A70FF2845D80F2302
:1054C00007261C001840FF2D58D8FF222D0115403B
:1054D0002843F025E0222C43F025D20232432D034D
:1054E0002B43394D07262F683D00AC352D886E4380
:1054F000350001963E6AAD192E68002EFCDA334D58
:105500002E78334D002E03D0324EAE59002E50DA95
:10551000314E32493160324E32493160A321C900E7
:105520006E58A6430643304C6E50285998430243A8
:1055300000202A512D4B009A1A60264BEA503B6AF4
:10554000019AD31800225A60FEBD294B984205D813
:105550000F231840060000242000B4E7254B060A5C
:10556000984204D8FF2304011C402643F3E7F023AC
:1055700000021B01184006431F4BECE71C4A9542F2
:1055800005D82A04F0252D032A403243A8E72A0A29
:1055900012043243174EB54207D8F0262D053604C3
:1055A00035402A43FF252D049AE72D062A43134D43
:1055B00096E71348C3E71248C6E7C0460F06000047
:1055C000FFFFFF0028070E0818090E0834070E0811
:1055D000000026401C050000080126401F1F000097
:1055E000040126403D3D00001405000024070E087C
:1055F000FF040000FF0500000F0F000000000F0F68
:1056000001004A00F8B5144B984219D90027134BF2
:10561000C018F6213F23124D124CF6302E59490086
:105620001E4000F0D9FF321A002F00D032183F215F
:105630002B590A408B4313432B51002F09D0F8BD3F
:10564000094B984204D8EE33FF33181A0127E0E7DC
:1056500000204042F3E7C046EC8100000080FFFFDD
:105660000000264018FF0000137E0000E02210B565
:105670000124094B80009200C018835880589B0673
:105680009B0F9C400F231840FFF762FE6308181819
:10569000210000F0A1FF10BD00002640144B30B5E2
:1056A0001A680724130028331B781F2B15D883088A
:1056B0001D00A5432C1E0FD103342040A040814083
:1056C00012689B002032D3180A00FF2181401C6819
:1056D000624011406140196030BD802320401B06AC
:1056E000184380239B011268C91889008850F3E78A
:1056F00018090E08064B9A680300064810339B00F1
:10570000824202D1985899507047034AD058FBE71B
:1057100000ED00E000000E0800040010F8B50600DF
:105720000D0000283AD00023C05E002828DB7188D5
:10573000FFF7B4FF0024FF22032794460023F05E06
:10574000716883B21F40FF006646BA40890131404C
:10575000D243B940002815DB114E83089B009B19EA
:10576000C026B6009F593A40114399510D4B9A6893
:105770000D4B9A4202D12900FFF7BCFF2000F8BD73
:105780000A4CD8E70F263340083B064E9B089B0087
:105790009B19DE6932401143D961E7E7034CEDE71D
:1057A00000E100E000ED00E000000E0801005600FE
:1057B00070B5802504002D02AC4205D8064B186850
:1057C0006043FAF781FE70BD044B1868FAF77CFE5F
:1057D000034BE418F0E7C046F4000E08F0000E0892
:1057E0000080FFFF10B5034B1B785843FAF76CFE9F
:1057F00010BDC046F8000E088022054B12069A64C0
:10580000986C044BC043C0171840034BC018704736
:1058100000002740FDFFB9FF030046008022054B32
:10582000120198585B68DBB2002B02D08023DB02A8
:105830001843704700002640FEE7000002680A4B4C
:1058400010B51A6042685A6082689A60C268DA606D
:1058500002691A6142695A6182699A61C269DA61B0
:10586000FFF7EAFF10BDC046D0050E08F0B51922BB
:10587000002800D14B322A4B8A4292411B68524287
:105880001C00A43424881D68671903253E68AE43B4
:1058900016433E601E68A4192768224E37402760D1
:1058A0001C00A63424881E68A7193E68AE43324304
:1058B0003A601A681B4EA218146826401660002829
:1058C0000ED00020102904D9213088428041404266
:1058D00001300F225B681968914308431860F0BDDE
:1058E0001A00513212788A42F3D21A0052321278D8
:1058F00001208A42EDD21A005332127800188A42EF
:10590000E7D21A005432127828008A42E1D21A00F3
:10591000553210788842804140420430D9E7C04671
:1059200018090E08FFFCFFFFB0235B059A89002AC7
:1059300002D0988980B2704780204000FBE70000C9
:10594000074A084BD058B022E8235205DB00D35C4D
:105950001F221040C01A431E9841C0B27047C04673
:10596000000026401CFF00000120024B1B68DB0DDD
:10597000984370470000264070B5FFF7D5FF80239D
:10598000194A5B00984215D111680F240B000222BE
:10599000943318680B6818180368A3431343036013
:1059A000080098300B6801685B181968A1430A4326
:1059B0001A6070BDB02412680C4B11006405E358E6
:1059C0000B4D94312B40C02510680968AD0041187B
:1059D0000868284003430B601100983113680A6877
:1059E0009B18044AA258E3E718090E08481800005B
:1059F000FFFCFFFF4418000070B5FFF795FF802300
:105A00001A4A5B00984215D111680F240B0003223B
:105A1000943318680B6818180368A3431343036092
:105A2000080098300B6801685B181968A1430A43A5
:105A30001A6070BDB02412680D4B11006405E35864
:105A40000C4D94312B40C02510680968AD004118F9
:105A50000868284003430B601100983113680A68F6
:105A60009B18C1225201A258E2E7C04618090E084D
:105A700024180000FFFCFFFF10B5FFF755FF80233F
:105A8000124A5B0098420DD1136811491A009432F2
:105A900012681B689B181A681140C022D2010A4381
:105AA0001A6010BDB02112680A4B4905CB5811008D
:105AB000094894310340C0200968126880005218D8
:105AC000116801400B431360EBE7C04618090E084C
:105AD000FF8FFFFF1C180000FFFCFFFF70B5FFF7F2
:105AE00023FF8023154A5B0098420DD113681449A7
:105AF0001A00943212681B689B181A6811408022A1
:105B0000D2010A431A6070BDB02412680D4B110017
:105B10006405E3580C4D94312B40C025106809688A
:105B2000AD0041180868284003430B60110098310C
:105B300013680A689B18054AA258E3E718090E087B
:105B4000FF8FFFFF50180000FFFCFFFF4C18000004
:105B5000F8B51F4FC0253B682D011A0094321B6811
:105B600012689B181E68FFF7DFFE340080232C406C
:105B70005B0098420FD10020FFF7FEF8B0235B05D1
:105B80005A78002A03D05A780123222A01D84342A6
:105B900043411800F8BD3B680E4F190094311A6854
:105BA000086812181068384010601A6808681218DF
:105BB00028001768B043384310601B680A689B18B8
:105BC00018682840001B431E9841C0B2E2E7C04657
:105BD00018090E08FFF3FFFF10B50D4C23689B0654
:105BE00013D5FFF7C1FE226800280CD0094B1343E0
:105BF00023600120FFF7F6FD802300202268DB05EB
:105C00001343236010BD044BF1E70448FAE7C04694
:105C100000002640000004170000041604004200A3
:105C200010B5FFF7A1FE104C236800280DD00F4AD5
:105C3000134023600820FFF7D5FD64232268002A63
:105C400007DB002B03D10A480DE00A4AF0E7013BCD
:105C5000F4E7002BF7D02368074A012013402360A4
:105C6000FFF7C0FD002010BD00002640FFFFFBAC89
:105C700002004200FFFFFBADFFFFFFFB10B50C4B26
:105C80001B6843331B78002B11D08022094BD205AF
:105C90005969114202D159690A435A6180229620FA
:105CA000996912060A439A618000FFF79BFD10BDB7
:105CB00018090E080000264070B50C4B1B684333D2
:105CC0001B78002B11D00722094DAC691440A0426B
:105CD0000BD0AB69934302401343AB61002904D05E
:105CE000A04202D9C820FFF77DFD70BD18090E083B
:105CF000000026407FB5274B86000D00F45804298C
:105D000001D0012927D100200FE0A3682B420BD13D
:105D1000E36829001A685B6802920193039302A862
:105D2000236898471C4B1C606469002C0BD01B4BEC
:105D30009842EAD1012DE8D1174B18481A68184B40
:105D40009A5104B070BD012DFBD1144B9842F3D091
:105D5000134B9C51F5E7022906D10F4B1B68181E07
:105D6000EFD01C6903E01C006369002BFBD100200D
:105D7000002CE6D0A3682B4209D1E36829001A68F9
:105D80005B6802920193039302A8236898472469F1
:105D9000EEE7C04678070E0874070E08FF004200C1
:105DA00060070E08B02370B55B055A780400212502
:105DB000002A01D05D78EDB2FFF7B6FD06000020A5
:105DC000FEF7DAFF8023ADB25B00002811D19E42BE
:105DD00011D1222D0FD880251E4B6D041B6824067F
:105DE00059681D4B2C40CA581C4D2A401443CC50B6
:105DF00070BD9E4228D0174A1268156A9E420ED185
:105E000062426241FF2352429A43154BD21801214C
:105E10002800FBF7D9FF002808D01248E8E76242C3
:105E20006241012352429A430F4BEFE7094B1B6833
:105E3000B0331B68EB181A68002AFCDBEB68002003
:105E40001B0EA02BE9D1D3E7222DE6D9014B1B680D
:105E50001D6AD5E718090E0818F00000FFFFFFFEC5
:105E600001010030040042000300000C70B5050081
:105E7000FFF76EFE002834D0FAF72FFB0600022D44
:105E800017D10120FFF78EFF041E0DD1FFF774FD1F
:105E9000072215494B6993432A4013434B61022D56
:105EA00015D1FFF7E9FD00243000FAF71AFB2000B6
:105EB00070BD07220C4934204B6993431A00032319
:105EC00013434B61FFF78EFCFFF708FEE0E79120DC
:105ED000FFF788FCFFF790FD0020FFF763FF040049
:105EE000E2E7024CE3E7C046000026400300420020
:105EF000F7B50700FFF72CFE002843D0FAF7EDFABC
:105F0000B0230190204D214A5B05002F1CD1AF50DA
:105F1000E8220120D2009C5CFFF744FFE4B2061E99
:105F20000DD1FFF729FD1F21194A0C40AB588B43B7
:105F30001C43AC50002F1BD1FFF79EFD3E00019883
:105F4000FAF7CFFA3000FEBD124903205958A95084
:105F5000114A0F499C5C1F226B58E4B293431A000C
:105F60000B2313436B50FFF73DFCFFF7B7FDDAE758
:105F70000720FFF737FCFFF73FFD0020FFF712FF78
:105F80000600DCE7054EDDE700002640307F00001C
:105F90001CFF000010180000410700000300420031
:105FA000F8B50500FFF7E0FC002857D0FAF795FA9E
:105FB0000600022D3CD1FFF7C3FC00282ED11F2282
:105FC0002C482D49435893431A000B231343435045
:105FD0000920FFF707FCE023264FDB033A68E120A6
:105FE000134307223B607B69154093431D43802385
:105FF0007D617A69DB0513437B6180237A691B0627
:1060000013437B618000FFF7EDFB802300243A6897
:106010001B0413433B60194BFC5004E00020FFF7C6
:1060200067FF041ECBD03000FAF75BFA2000F8BD02
:10603000052D11D1FFF784FC012807D11F220D483F
:106040000D49435893431A001B23BFE70120FFF774
:106050004FFF041EF2D0E6E7094CE4E70722054BA8
:1060600004005B6913409D42E0D02800FFF7FEFE6C
:106070000400DBE7000026401CFF0000307F00002A
:1060800003004200194B1B68190004C9C96F51185D
:106090000968016219000831C96F5218126842621A
:1060A0001A0042321278002A1FD09A68E032126831
:1060B000D2061AD5F222DB68D2019A580260F02289
:1060C000D2019A5842600A4A9A588260094A9A58FC
:1060D000C260094A9A580261084A9A584261084ABD
:1060E0009A588261074A9B58C361704718090E0885
:1060F00004780000087800000C7800001078000098
:106100001478000018780000194B1B681A1D1968D4
:10611000D26F8A18016A11601A0008321968D26FAA
:106120008A18416A11601A0042321278002A1ED081
:106130009A68E0321268D20619D5F0224168DB680D
:10614000D201995081680B4A9950C1680A4A995006
:1061500001690A4A99504169094A99508169094A75
:106160009950C169084A99500168E83299507047BE
:1061700018090E0804780000087800000C78000068
:10618000107800001478000018780000B023F7B5EC
:106190005B055A7807002126002A01D05E78F6B206
:1061A000624D6B68002B00D07CE0FAF796F96B68C3
:1061B0000090002B00D088E05D4C22681300AC33C7
:1061C000198807234B43126A9B181A68002AFCDAC5
:1061D000DB68DA0020D51B0F1B0756480193FFF739
:1061E00051FF5549212E00D074E090202268000113
:1061F000131DDC6F13681C1923680B4003432360D5
:10620000130008331268DB6FD3181A681140084373
:106210001860484B019A13438022454E920531681D
:1062200013430A00AC321088072200244243096A53
:106230005218D36054605368FFF776FB80235B00ED
:1062400098425CD1380000F0A3FD32681300AC33F3
:10625000198807234B43126A9B181A68002AFCDA34
:10626000DF68FB0003D538010009FFF74DFF334B12
:1062700032681F401300AC33198807234B43126A5E
:1062800000989B180022DF605A60FAF72AF9002C68
:106290000FD16B68002B03D008210120FFF72AFDE6
:1062A0002000FEBD01210800FFF724FD041E00D1DF
:1062B0007BE76B68002B03D002210120FFF71AFD5A
:1062C0001F4B9C42ECD01F4CEAE704210120FFF752
:1062D00011FD71E7802220685200031DDC6F036806
:1062E0001C1923680B401343236003000833006824
:1062F000DB6FC318186801400A431A6089E73268E7
:106300001300B0331B68126A9B181B68002B0ADB52
:1063100004230D4A11690B431361012F01D030BFD3
:1063200093E720BF91E7064C8FE7C04678070E0839
:1063300018090E0838070E08FF00FFFFFFFFFFDFF8
:1063400005004200FF00420000ED00E0C023044AC7
:106350005B00D058800F431E9841C0B27047C046C2
:1063600000002640C0228020064952008B58C005FC
:106370009B009B0803438B50802388581B060343D4
:106380008B5070470000264037B562B680206A46C1
:1063900001A94000FBF758FB0F4D00230F4A2900CD
:1063A0000198FAF7BDFC2B0038331B78002B0FD077
:1063B0008022EB6BD200ED6A9C1806210E20FEF7BE
:1063C000BDFC2A0020000121FBF7E0FB00203EBDC0
:1063D00080226B695202EEE71C0A0E08A40B0E081D
:1063E00010B50020FBF7E8FD10BD704710B5002088
:1063F000FFF73CF9002829D0154B1860154B1B6896
:106400001A1D1C68D36FE4182168090E013100F0D1
:10641000E3F8114B18602168090AC9B2013100F094
:10642000DBF80E4B441E18600D49200000F0D4F834
:10643000FA210C4B013018708900200000F0CCF8D4
:10644000094B01301860094BC003186010BDC046ED
:10645000E8000E0818090E08EC000E08E4000E080B
:1064600040420F00F8000E08F4000E08F0000E087D
:1064700010B52148FBF7CAFBB022E02130201F4CA9
:10648000D200A35889005B005B08A3506358834384
:10649000635080235B04A350194B1A4AE250A02298
:1064A00004339201E250FF22174BE250FFF75AFFEC
:1064B000C02201215200A3588B43A350FFF795FF40
:1064C000FFF794FF114B03201A681300AC331988AF
:1064D00007234B43126A80219B180022DA605A601E
:1064E0000B4AFBF7B1FD0B48FBF78CFC0A48FBF7A6
:1064F000BDFCFDF789F810BD70700010000026404B
:1065000084050000010002008C05000018090E0837
:106510000C0000088C070E08247100109023034A19
:106520005B01D058032318407047C046000020404C
:1065300010B59024F9F7D1FF074B64011A590749A8
:106540001140074A0A431A51102259681142FCD0DF
:10655000F9F7C7FF10BDC04600002040FCFF000057
:106560000100FA05F8B590250E4C6D010700F9F70A
:10657000B4FF63590600DB439B0701D1FFF7D8FF47
:1065800080239B00E7506359074A1A40074B134387
:106590006351102362681A42FCD03000F9F7A1FF62
:1065A000F8BDC04600002040FCFF00000300FA05D3
:1065B00002B4714649084900095C49008E4402BC96
:1065C0007047C04603B47146490840004900095A63
:1065D00049008E4403BC7047002243088B4274D3A9
:1065E00003098B425FD3030A8B4244D3030B8B42D4
:1065F00028D3030C8B420DD3FF22090212BA030CDD
:106600008B4202D31212090265D0030B8B4219D3BD
:1066100000E0090AC30B8B4201D3CB03C01A5241DD
:10662000830B8B4201D38B03C01A5241430B8B4225
:1066300001D34B03C01A5241030B8B4201D30B030E
:10664000C01A5241C30A8B4201D3CB02C01A524135
:10665000830A8B4201D38B02C01A5241430A8B42F8
:1066600001D34B02C01A5241030A8B4201D30B02E1
:10667000C01A5241CDD2C3098B4201D3CB01C01AFB
:10668000524183098B4201D38B01C01A5241430905
:106690008B4201D34B01C01A524103098B4201D3F3
:1066A0000B01C01A5241C3088B4201D3CB00C01A60
:1066B000524183088B4201D38B00C01A52414308D8
:1066C0008B4201D34B00C01A5241411A00D20146FD
:1066D000524110467047FFE701B5002000F006F870
:1066E00002BDC0460029F7D076E770477047C04624
:1066F000002B11D1002A0FD1002900D1002802D08F
:106700000021C943081C07B4024802A140180290A6
:1067100003BDC046D9FFFFFF03B4684601B5029828
:1067200000F030F8019B9E4602B00CBC7047C0469A
:10673000F0B5CE46474615042D0C2E0080B5070453
:10674000140C3F0C9946030C7E435D43674363433F
:106750007F19340CE4199C46A54203D980235B02BF
:106760009846C4444B4643435143250C3604654484
:10677000360C2404A4195B19591820000CBC90464F
:106780009946F0BDF0B54F464646D646C0B5040022
:1067900082B00D00914698468B422FD82CD04146AE
:1067A000484600F0CFF829000600200000F0CAF8A3
:1067B000331A9C46203B9A4600D576E04B4652461B
:1067C00093401F004B46624693401E00AF4228D8BC
:1067D00025D05346A41BBD41002B00DA7BE00022EC
:1067E0000023009201930123524693400193012319
:1067F00062469340009318E08242D0D900220023E1
:10680000009201930A9B002B01D01C605D600098F0
:10681000019902B01CBC90469946A246F0BDA34225
:10682000D7D900220023009201936346002BE9D0C0
:10683000FB079846414672080A437B0866460EE00D
:10684000AB4201D1A2420CD8A41A9D4101202419C7
:106850006D410021013E24184D41002E06D0AB426F
:10686000EED9013E24196D41002EF8D1009801990E
:10687000534600196941002B23DB2B005246D340BD
:106880002A006446E2401C0053461500002B2DDB15
:1068900026005746BE40330026006746BE40320001
:1068A000801A994100900191ACE7624620239B1A1F
:1068B0004A46DA406146130042468A4017001F43A9
:1068C00080E7624620239B1A2A0066469A402300EE
:1068D000F3401343D4E76246202300219B1A002291
:1068E000009101920122DA40019280E72023624662
:1068F00026009B1ADE402F00B0466646B74046464B
:106900003B003343C8E7C0461C2101231B049842C7
:1069100001D3000C10391B0A984201D3000A083930
:106920001B09984201D30009043902A2105C4018E7
:106930007047C0460403020201010101000000008B
:106940000000000010B5002903D1FFF7DDFF203063
:1069500002E0081CFFF7D8FF10BDC046EC3000680D
:106960007047000010B5034B0100186800F07CF878
:1069700010BDC046FC000E0810B5034B010018689E
:1069800000F028F810BDC046FC000E0882B00029B7
:1069900000D101A9101E06D0002B06D013780B6081
:1069A0001078431E984102B0704702204042FAE737
:1069B000002310B59A4200D110BDCC5CC454013301
:1069C000F8E703001218934200D1704719700133A1
:1069D000F9E7000070B50500002910D00C1F2368EE
:1069E000002B00DAE418280000F0ACF91D4A136807
:1069F000002B05D163601460280000F0A4F970BD7D
:106A0000A34209D9216860188342F3D118685B68F2
:106A100041182160EEE713005A68002A01D0A24213
:106A2000F9D919685818A0420BD1206809185818CC
:106A300019608242E0D110685268411819605A60AA
:106A4000DAE7A04202D90C232B60D5E72168601851
:106A5000824203D1106852684118216062605C6014
:106A6000CAE7C0460C090E08032370B5CD1C9D4330
:106A7000083506000C2D1ED20C25A9421DD8300069
:106A800000F060F9254A14682100002919D1244C2E
:106A90002368002B03D1300000F044F82060290067
:106AA000300000F03FF8431C2BD10C233000336042
:106AB00000F049F903E0002DDFDA0C2333600020F9
:106AC00070BD0B685B1B19D40B2B03D90B60CC1862
:106AD000256003E04B688C420DD11360300000F05C
:106AE00032F9200007220B30231D9043C31AE7D050
:106AF0005A42E250E4E763600C00EFE70C0049689B
:106B0000C3E70323C41C9C43A042E1D0211A3000F8
:106B100000F008F8431CDBD1C7E7C0460C090E089B
:106B200010090E08002370B5064C0500080023600C
:106B300000F00AF9431C03D12368002B00D02B601E
:106B400070BDC046AC0B0E08C9B20378002B04D050
:106B50008B4200D170470130F7E74B42594149421F
:106B60000840F7E702780B78002A03D001300131A2
:106B70009A42F7D0D01A704703000A7801311A7090
:106B80000133002AF9D17047002330B59A420AD068
:106B9000013AC45CCD5CAC4204D1934202D00133D3
:106BA000002CF6D1631B180030BD0000F0B51F00AB
:106BB0000E008DB00B900291039212983478FFF77B
:106BC000CDFE082200194378751C134053D12D2C9B
:106BD00053D17478B51C01330193002F00D18AE0A2
:106BE000102F0AD1302C08D120222B789343582B18
:106BF00000D07AE010276C780235019B002B41D140
:106C0000013B04933E4B05933A00FB17049805990A
:106C10000893FFF76DFD002309900E00002000216E
:106C20000A922200303A092A31D81400A7423DDDE9
:106C30005A1C1DD0B14236D802D1099B984232D895
:106C4000099B834206D18E4204D101230A9A5B42FA
:106C5000A2420DDB0B00020008993800FFF768FD27
:106C6000E31706940793069B079CC0186141012314
:106C70002C780135D5E72E009FE72B2CACD1B51C25
:106C80007478A9E70023049380231B06BBE7220046
:106C9000413A192A01D8373CC8E72200613A192A3B
:106CA00004D8573CC2E701235B42E1E75A1C09D1F3
:106CB0000B9A23331360039B04980599002B0ED184
:106CC0000DB0F0BD019A002A04D006000F0000218B
:106CD0007042B941039A002AF2D0002B01D06B1EFA
:106CE0000293039B029A1A60EAE73024002F00D037
:106CF00083E7082781E7302C00D175E70A277CE776
:106D0000FFFFFF7F37B51300064A05001068046ACD
:106D1000002C00D1044C0A0000942900FFF746FF24
:106D200003B030BDFC000E0860010E080B1E04D03D
:106D3000FF2A04D98A2303608B3B180070470A702E
:106D40000123FAE770477047044A1368002B00D10B
:106D5000034B1818106018007047C04614090E083D
:106D6000B00B0E08F8B5C046F8BC08BC9E4670478C
:106D7000F8B5C046F8BC08BC9E467047000000004D
:106D800001B40248844601BC604700BFD5020E082A
:106D900001B40248844601BC604700BF99040E0854
:106DA0004142434445464748494A4B4C4D4E4F505B
:106DB0005152535455565758595A61626364656627
:106DC0006768696A6B6C6D6E6F70717273747576DB
:106DD0007778797A30313233343536373839006E56
:106DE000756C6C0066616C73650074727565007219
:106DF00065736F757263657300424F4F5400555051
:106E0000475241444500616464726573730073695D
:106E10007A65006C61756E6368006163715F7769A4
:106E20006E006D756C74695F696D616765006D6F8B
:106E30006E6F746F6E696300656E63727970740053
:106E4000656E63727970745F6B65795F6964006207
:106E500061636B757000626F6F745F617574680059
:106E6000736D69665F696400726570726F677261E5
:106E70006D00737461727400726570726F766973FD
:106E8000696F6E00626F6F745F6C6F616465720032
:106E90006B6579735F616E645F706F6C6963696560
:106EA00073006D34007065726D697373696F6E0085
:106EB000636F6E74726F6C006B65790070726573CE
:106EC000656E74006669726D7761726500636572E4
:106ED0007469666963617465006F70656E006469EA
:106EE0007361626C656400656E61626C656400610B
:106EF0006C6C6F77656400646562756700626F6FC4
:106F0000745F7570677261646500747970650061A3
:106F100072726179006974656D73006E756D62657A
:106F20007200696E746567657200626F6F6C65618F
:106F30006E00737472696E67006D6178696D756D4E
:106F4000006D696E696D756D00464C4153485F5028
:106F500043315F53504D00464C4153485F504332DC
:106F600000464C4153485F50433300464C41534820
:106F70005F50433400464C4153485F4D41494E5F9A
:106F8000434F444500464C4153485F4D41494E5F95
:106F9000584F00464C4153485F4D41494E5F444174
:106FA000544100464C4153485F5355504552564951
:106FB000534F525900464C4153485F574F524B5F15
:106FC00053454355524500464C4153485F574F5235
:106FD0004B005352414D5F5043305F505249560071
:106FE0005352414D5F5043305F5055420053524120
:106FF0004D5F53504D5F50524956005352414D5FC3
:1070000053504D5F505542005352414D5F504331F4
:107010005F50524956005352414D5F5043325F50CA
:10702000524956005352414D5F5043335F505249CD
:1070300056005352414D5F5043345F505249560001
:107040005352414D5F4D41494E005352414D5F44B3
:10705000415000534D49465F434F444500534D490D
:10706000465F584F00534D49465F4441544100002C
:10707000000020400000244000000040000000000C
:1070800000002340000030400000314000009F40DD
:10709000000022400000104020202020201010106E
:1070A0001D1D800017007500FF0306020600360450
:1070B000102000007FC0000000040000000000005D
:1070C0000019324B647D00804000080B1000000066
:1070D0000000FF012002001F00800004FF081018BC
:1070E000001000140018001C4044484C50000000E0
:1070F0000810000008000000040000000410000058
:107100000012000004210000002100000016000011
:1071100040114002C41300138013A013200000008C
:107120001C0000000300000001000000010000003E
:1071300000000000050360000400000001000000E2
:1071400000000000010000000604600008000000CC
:10715000EC080E08E16300104300504F53495800FB
:107160002E00002020202020202020202828282831
:107170002820202020202020202020202020202007
:107180002020208810101010101010101010101057
:107190001010100404040404040404040410101067
:1071A0001010101041414141414101010101010113
:1071B00001010101010101010101010101011010A1
:1071C00010101010424242424242020202020202E7
:1071D0000202020202020202020202020202101073
:1071E000101020000000000000000000000000005F
:1071F000000000000000000000000000000000008F
:10720000000000000000000000000000000000007E
:10721000000000000000000000000000000000006E
:10722000000000000000000000000000000000005E
:10723000000000000000000000000000000000004E
:10724000000000000000000000000000000000003E
:10725000000000000000000000000000000000002E
:08726000000000000000000026
:087268001CF5FF7F010000008E
:107270000004001000000E08800000009072001052
:0872800080000E08500500001B
:08728800F0050E08C00500002E
:107290007969001065690010496F0010576F001080
:1072A000616F00106B6F0010756F0010856F00101C
:1072B000936F0010A36F0010B56F0010C76F001020
:1072C000D26F0010E06F0010ED6F0010FB6F001028
:1072D000087000101670001024700010327000103A
:1072E000407000104A700010537000105D70001064
:1072F0006570001000093D0000127A0000093D0091
:107300000000D007A00F00000400000000010E08DC
:10731000000000000000000000000000000000006D
:10732000000000000000000000000000000000005D
:10733000000000000000000000000000000000004D
:10734000000000000000000000000000000000003D
:10735000000000000000000000000000000000002D
:10736000000000000000000000000000000000001D
:1073700043000000000000000000000000000000CA
:1073800000000000000000000000000000000000FD
:1073900043000000000000000000000000000000AA
:1073A00000000000000000000000000000000000DD
:1073B000430000000000000000000000000000008A
:1073C00000000000000000000000000000000000BD
:1073D000430000000000000000000000000000006A
:1073E000000000000000000000000000000000009D
:1073F000430000000000000000000000000000004A
:10740000000000000000000000000000000000007C
:107410004300000000000000000000000000000029
:10742000000000000000000000000000000000005C
:107430004300000000000000000000000000000009
:10744000000000000000000000000000000000003C
:107450002D6D00108D690010000000006271001099
:107460006071001061710010617100106171001095
:107470006171001061710010617100106171001084
:107480006171001061710010FFFFFFFFFFFFFFFF40
:10749000FFFFFFFFFFFF0000010041534349490088
:1074A00000000000000000000000000000000000DC
:1074B0000000000000000000000041534349490063
:1074C00000000000000000000000000000000000BC
:1074D000000000000000000000000000A9040010EF
:1074E00081040010024A1368002BFCDB7047C04681
:1074F0000001264010B54378FF2B0BD1032000F08C
:107500004FF9C3685A680123116819431160116863
:107510001942FCD110BD80B230B5C00020D0114B53
:1075200007221C682300AC331B885A43236AD318F4
:1075300019680029FCDA3E210B4B062519600B4B1C
:107540000B491960A3210B4BC9005D500A495850E3
:107550005858206A1218002050605A58002AFCDA45
:1075600030BDC04618090E08040126400801264017
:107570001E1F0000000026401C050000F7B500900B
:107580000020019100F00CF93E4D06002B681A0016
:107590004C33B03214681B780419002B5AD000F019
:1075A000EFF8070003281BD000F00AF9364A374BE2
:1075B0000500D358002B3EDA354A0121300000F097
:1075C000E7F8002837D10198FFF7A5FF009B002BB3
:1075D0003ED02368002BFCDB00F0CAF804002BE04F
:1075E000062000F0DDF82B68B0331B68C018036874
:1075F000002B02DA274C2000FEBD002000F098F896
:10760000254B9842F6D00023244A19001268012025
:1076100000F096F80025A842ECD1002000F088F890
:107620001D4A1F4B904203D09D42E3D00135F4E741
:107630009D42B9D1DEE7174C032F05D1012100206F
:1076400000F0B6F80028F9D1280000F0C1F8D2E720
:10765000144CF1E700F0B4F80D4A050001213000A8
:1076600000F096F8002809D1009B002B08D0236871
:10767000002BFCDB00F07CF80400E5E7054CE3E7B9
:10768000084CE1E718090E08000026401C05000020
:1076900010060E08050052000101880020060E08A1
:1076A000F0490200010050001A4BF7B51B681A4A56
:1076B0005C68042311690B431361012828D030BF93
:1076C0002300FC335B6F002B21D100F049F8A3208D
:1076D000124B1349134AC0000F681E5815680195D4
:1076E000114D0D6006251D503E2010600F483E359F
:1076F0001D501D58002DFCDA0120FC3460670F601E
:10770000A321C9005E50019B136000F021F8F7BD72
:1077100020BFD5E718090E0800ED00E00000264064
:1077200008012640040126401E1F00001C05000021
:1077300001B40248844601BC604700BF0521001027
:1077400001B40248844601BC604700BFD51E00104A
:1077500001B40248844601BC604700BF3B4D0010A5
:1077600001B40248844601BC604700BF394D001097
:1077700001B40248844601BC604700BFDD1C001014
:1077800001B40248844601BC604700BF1D6500107B
:1077900001B40248844601BC604700BFC91D001007
:1077A00001B40248844601BC604700BF191C0010A8
:1077B00001B40248844601BC604700BF912000101C
:1077C00001B40248844601BC604700BFDB040010DE
:1077D00001B40248844601BC604700BFE3040010C6
:04000005100004EBF8
:00000001FF
